:020000040000FA
:06000000B4EF3BF012001A
:060008003FEF30F0120092
:0600180046EF30F012007B
:06002A0001004478000013
:0800300000030000A200000023
:08003800076A0D6A096A0A6AF1
:100040000B6A0C6A086A140E5AEC0AF005E1110EEC
:10005000E66E140EAAEC09F0900E5AEC0AF004E1D8
:10006000E66A900EAAEC09F0910E5AEC0AF004E14F
:10007000E66A910EAAEC09F00C0E5AEC0AF004E1C3
:10008000E66A0C0EAAEC09F00D0E5AEC0AF005E136
:10009000010EE66E0D0EAAEC09F0910E9EEC0AF030
:1000A000900E9EEC0AF0030E9EEC0AF0020E9EECFF
:1000B0000AF0010E9EEC0AF0000E9EEC0AF0040E0F
:1000C000E66E140E9EEC0AF0E66A44EC22F04D6EE9
:1000D000090EE15E4D500C0EA3EC09F00501256FF1
:1000E000E8CF07F5E8CF58F4E8CFD6F0E8500301A1
:1000F0003DEC0AF0A915F310A96F05012551030184
:100100003DEC0AF0C715F310C76F05012551030137
:100110003DEC0AF0E515F310E56F25C5DDF40D0E95
:10012000A3EC09F00501346FE8CF16F5E8CF7CF4B5
:10013000E8CFE5F0E85003013DEC0AF0B815F31004
:10014000B86F0501345103013DEC0AF0D615F310E8
:10015000D66F0501345103013DEC0AF0F415F3109C
:10016000F46F34C5ECF4170EA3EC09F00401636FCF
:10017000180EA3EC09F00401646F190EA3EC09F04A
:100180000401656F1A0EA3EC09F00401666F1B0EE3
:10019000A3EC09F00401876F1C0EA3EC09F0040125
:1001A000886F1D0EA3EC09F00401896F1E0EA3ECED
:1001B00009F004018A6F2B0EA3EC09F00301AC6F68
:1001C0002A0EA3EC09F00301AD6F290EA3EC09F090
:1001D0000301AE6FFF0EAE5D02E0AF6B01D0AF6901
:1001E0002F0EA3EC09F00301BB6F2E0EA3EC09F058
:1001F0000301BC6F2D0EA3EC09F00301BD6FFF0ED0
:10020000BD5D02E0BE6B01D0BE69A20EA3EC09F099
:100210000301CA6FA10EA3EC09F00301CB6FA00E7E
:10022000A3EC09F00301CC6FFF0ECC5D02E0CD6BB7
:1002300001D0CD69A50EA3EC09F00301D96FA40E7E
:10024000A3EC09F00301DA6FA30EA3EC09F003019C
:10025000DB6FFF0EDB5D02E0DC6B01D0DC69A80E1A
:10026000A3EC09F00301E86FA70EA3EC09F003016A
:10027000E96FA60EA3EC09F00301EA6FFF0EEA5D39
:1002800002E0EB6B01D0EB69AB0EA3EC09F00301CC
:10029000F76FAA0EA3EC09F00301F86FA90EA3EC07
:1002A00009F00301F96FFF0EF95D02E0FA6B01D06E
:1002B000FA69200E5AEC0AF008E1210E5AEC0AF015
:1002C00004E1220E5AEC0AF065E007800201BE6BE1
:1002D000BF6B50EC0AF0200EA3EC09F02A6E210E41
:1002E000A3EC09F02B6E220EA3EC09F02C6E16EC99
:1002F0000AF04DE324EC0AF04AE3FA0ED8802F54BA
:10030000000E305403E32FC0BAF205D00D8830EC54
:100310000AF04DC0BAF2040E0201BA5D12E20D8479
:10032000BA51030A09E0010A03E0030A01E078D0A8
:10033000600E156EEA0E03D0400E156E9C0E166E02
:100340006FD0BA417F0BC06FBA51E840E8403F0B15
:10035000C36FBA51E840E840E8401F0BC66FBA3996
:100360000F0BC96FBA51E00BE838E840CC6F060EAE
:10037000BAC2E7FF070B04E0E742E79EE806FCE1AC
:10038000E7500201CF6FBA45010BD26F49D002018D
:10039000BA6B46D0B40E5AEC0AF00CE1B50E5AEC2A
:1003A0000AF008E1B60E5AEC0AF004E1B70E5AEC76
:1003B0000AF032E007860201BA6B300E286EB40EE6
:1003C000A3EC09F0296EB50EA3EC09F02A6EB60E67
:1003D000A3EC09F02B6EB70EA3EC09F02C6E1DEC0C
:1003E0000AF013E32AEC0AF010E30D842FC0BEF2EA
:1003F00030C0BFF2B7EC09F03FC0E9F240C0EAF20A
:1004000041C0EBF242C0ECF203D00201BE6BBF6B05
:100410000401856B866B04D00201BA6BBE6BBF6BA7
:10042000240E5AEC0AF008E1250E5AEC0AF004E119
:10043000260E5AEC0AF065E007820201BC6BBD6B28
:1004400050EC0AF0240EA3EC09F02A6E250EA3EC62
:1004500009F02B6E260EA3EC09F02C6E16EC0AF0B8
:100460004DE324EC0AF04AE3FA0ED8802F54000E34
:10047000305403E32FC0BBF205D00D8A30EC0AF0F4
:100480004DC0BBF2040E0201BB5D12E20D86BB51F2
:10049000030A09E0010A03E0030A01E078D0600ED4
:1004A000176EEA0E03D0400E176E9C0E186E6FD0BA
:1004B000BB417F0BC16FBB51E840E8403F0BC46FAD
:1004C000BB51E840E840E8401F0BC76FBB390F0B3A
:1004D000CA6FBB51E00BE838E840CD6F060EBBC2D7
:1004E000E7FF070B04E0E742E79EE806FCE1E75080
:1004F0000201D06FBB45010BD36F49D00201BB6B2A
:1005000046D0B00E5AEC0AF00CE1B10E5AEC0AF0EB
:1005100008E1B20E5AEC0AF004E1B30E5AEC0AF00C
:1005200032E007840201BB6B300E286EB00EA3ECE4
:1005300009F0296EB10EA3EC09F02A6EB20EA3ECFD
:1005400009F02B6EB30EA3EC09F02C6E1DEC0AF033
:1005500013E32AEC0AF010E30D862FC0BCF230C082
:10056000BDF2B7EC09F03FC0E5F240C0E6F241C091
:10057000E7F242C0E8F203D00201BC6BBD6B04019C
:10058000616B626B04D00201BB6BBC6BBD6BCD9029
:10059000CD82CD94CD96CF0ECD140009CD6E3F0EF9
:1005A000CD148009CD6E0DA603D0CF68CE6802D0E1
:1005B000CF6ACE6AB190B182B194B196CF0EB11428
:1005C0000009B16E3F0EB1148009B16E0DA403D0C5
:1005D000B368B26802D0B36AB26AB79EB68E876A51
:1005E000F90EA96EFC0E88140309886E870E881414
:1005F0000009886E88840DA402D0A08201D0B68044
:100600000DA602D09D8001D0A3849F90A292A584C4
:10061000B880B88EB68ED08E99920F0150815083DB
:1006200050955087BBC251FF526B99844D814D83C9
:100630004D954D87BAC24EFF4F6B6CEC0AF0B75127
:100640000001B397010B01E0B3870201B75100012C
:10065000B399020B01E0B38941EC0AF0B495040BA5
:1006600001E0B48541EC0AF0B497080B01E0B487CF
:1006700041EC0AF0B499100B01E0B48941EC0AF0A6
:10068000B49B200B01E0B48B41EC0AF0B49D400B0D
:1006900001E0B48D41EC0AF0B49F800B01E0B48F0F
:1006A00045EC0AF0B595010B01E0B58545EC0AF083
:1006B000B597020B01E0B58745EC0AF0B599040B3C
:1006C00001E0B58945EC0AF0B59B080B01E0B58B5C
:1006D00045EC0AF0B59D100B01E0B58D45EC0AF034
:1006E000B59F200B01E0B58F0201B8510001B69310
:1006F000400B01E0B6830201B8510001B695800BB2
:1007000001E0B6850201B9510001BE91010B01E083
:10071000BE810001B551800B01E0010E516EB55153
:10072000400B01E0010E506EB551200B01E0010EAF
:100730004F6EB551100B01E0010E4E6EB551080B16
:1007400001E0010E4D6EB551040B01E0010E4D2488
:100750004E244F24502451240201B66FE850060A5B
:1007600019E0030A14E0010A0FE0070A0AE0010A8F
:1007700005E0030A12E10001320E0ED00001180E4E
:100780000BD00001100E08D000010C0E05D00001A6
:100790000A0E02D00001080ECA6F106A116A126AAE
:1007A000136A196A1A6A1B6A1C6A0201D76BD86B32
:1007B000D96BDA6BDB6BDC6BDD6BDE6BD56BD66B11
:1007C00012002350780DF3CF0EF0F4CF0FF002019A
:1007D000C251D880245406E2C251245E3C0E0E263B
:1007E000000E0F22C551D880245406E2C551245E64
:1007F0001E0E0E26000E0F22C851D880245406E289
:10080000C851245E0F0E0E26000E0F22CB51D88049
:10081000245406E2CB51245E070E0E26000E0F2252
:10082000CE51D880245406E2CE51245E040E0E260A
:10083000000E0F22D151D880245406E2D151245EFB
:10084000020E0E26000E0F22D451D880245405E249
:10085000D451245E0E2A000E0F2212000DA262D186
:100860000D920C50020A01E1AFD0050A01E1ACD0B3
:10087000060A03E0070A01E04DD107A075D00DA4D8
:100880001CD01B5016E01B50146E0201BA0502E189
:100890001490144214504D6E4E6A15C041F016C0AB
:1008A00042F0FEEC09F0D8900E360F36E806FBE178
:1008B00002D00E6A0F6A1B6A1DD01F50236E215092
:1008C000246EC0C2C2F2C3C2C5F2C6C2C8F2C9C257
:1008D000CBF2CCC2CEF2CFC2D1F2D2C2D4F271DF0F
:1008E0000DA808D0010E0F0B05E0D8900F320E3284
:1008F000E806FBE10E5010240501086F0F5011208F
:10090000096FD890093308330EC010F00FC011F0F2
:10091000020ED89008370937E806FBE10C0401E025
:10092000F9D0640ED8800E54000E0F5401E3F2D0BB
:100930000401632B000E642365236623635101E0E9
:10094000E9D063C4E6FF170EAAEC09F064C4E6FF21
:10095000180EAAEC09F065C4E6FF190EAAEC09F01E
:1009600066C4E6FF1A0EA4D007A6D4D00201000E7A
:10097000D880DD55000EDE5511E2DDC24DF0DEC23D
:100980004EF04F6A506AE9C23FF0EAC240F0EBC253
:1009900041F0ECC242F0EFEC09F002D0DF6BE06B0B
:1009A0000201DD6BDE6BDF51E3250401856F02017F
:1009B000E051E4210401866FD89086338533DFC28D
:1009C000E3F2E0C2E4F2A6D007A275D00DA61CD0D7
:1009D0001C5016E01C50146E0201BB0502E114907D
:1009E000144214504D6E4E6A17C041F018C042F0C8
:1009F000FEEC09F0D8900E360F36E806FBE102D087
:100A00000E6A0F6A1C6A1DD02050236E2250246E7D
:100A1000C1C2C2F2C4C2C5F2C7C2C8F2CAC2CBF2D6
:100A2000CDC2CEF2D0C2D1F2D3C2D4F2CADE0DAA68
:100A300008D0010E0F0B05E0D8900F320E32E806F9
:100A4000FBE10E5012240501176F0F501320186F91
:100A5000D890183317330EC012F00FC013F0020EE7
:100A6000D89017371837E806FBE1020E0C5C52E10C
:100A7000640ED8800E54000E0F544CE20401872BF4
:100A8000000E882389238A23875144E187C4E6FF27
:100A90001B0EAAEC09F088C4E6FF1C0EAAEC09F0B4
:100AA00089C4E6FF1D0EAAEC09F08AC4E6FF1E0EFB
:100AB000AAEC09F02FD007A42DD00201000ED88097
:100AC000DB55000EDC5511E2DBC24DF0DCC24EF00E
:100AD0004F6A506AE5C23FF0E6C240F0E7C241F01B
:100AE000E8C242F0EFEC09F002D0DF6BE06B0201EC
:100AF000DB6BDC6BDF51E1250401616F0201E0512A
:100B0000E2210401626FD89062336133DFC2E1F207
:100B1000E0C2E2F2020EE66EAFEC25F0E5520C50B8
:100B2000086E120000016B5148E0065046E1255066
:100B3000020B43E12550010B40E16BA107D069C0D6
:100B4000E6FF140EA1EC0AF06B9112006BA307D024
:100B500065C0E6FF900EA1EC0AF06B9312006BA546
:100B600009D00F0E00016815E66E910EA1EC0AF097
:100B70006B9512006BAB07D007C5E6FF0C0EA1EC1E
:100B80000AF06B9B12006BAD07D016C5E6FF0D0E89
:100B9000A1EC0AF06B9D12006BA707D025C5E6FFFC
:100BA0000C0EA1EC0AF06B9712006BA906D034C5AD
:100BB000E6FF0D0EA1EC0AF06B991200B7AE6BD0F8
:100BC000B79E092A140E095C33E3096A258625A815
:100BD00006D00A2A040E0A5C02E30A6A25980B2A48
:100BE000140E0B5C25E30B6A0D820C2A0C500A08CC
:100BF00002E2010E0C6E0DB40CD00C0403E0060EE4
:100C00000C5C07E11D501F6EB250216E1D6AB26A66
:100C1000B36A0DB60DD0020E0C5C03E0070E0C5C3F
:100C200007E11E50206ECE50226E1E6ACE6ACF6A39
:100C30000DA417D007A005D0FF0E195C12E2192AE7
:100C400010D007A60ED00201D62B040ED65D09E304
:100C5000D66BFF0ED95DFF0EDA5903E2D92B000ED9
:100C6000DA230DA625D007A205D0FF0E1A5C12E2EA
:100C70001A2A120007A41CD00201D52B040ED55D40
:100C800017E3D56BFF0ED75DFF0ED85911E2D72BB6
:100C9000000ED8231200B7A005D01D2AB26AB36A8D
:100CA000B7901200A4A404D01E2ACE6ACF6AA494DE
:100CB0001200A1A20DD019501B6E196AD9C2DDF223
:100CC000DAC2DEF20201D96BDA6BB368B268A192C4
:100CD0009EA00DD01A501C6E1A6AD7C2DBF2D8C281
:100CE000DCF20201D76BD86BCF68CE689E90120001
:100CF000D9CFE6FFE1CFD9FF0201F96BFE0EDBCFC2
:100D0000E6FFE66AB7EC3AF0E552E5520201F86F09
:100D1000FE0EDB2818DB0201F76FFE0EDB50020F20
:100D200012DB0201F66FFF0EF65DFF0EF759FF0EA4
:100D3000F859000EF95934E2300EFA6F300EFB6F9D
:100D4000300EFC6F300EFD6F100EF65D270E62DB6D
:100D500006E3100EF65F270E63DBFA2BF5D7E80EDD
:100D6000F65D030E57DB06E3E80EF65F030E58DB75
:100D7000FB2BF5D7640EF65D000E4CDB06E3640E2C
:100D8000F65F000E4DDBFC2BF5D70A0EF65D000E6C
:100D900041DB0EE30A0EF65F000E42DBFD2BF5D7BA
:100DA0002D0EFA6F2D0EFB6F2D0EFC6F2D0EFD6FAD
:100DB000FAC2E6FFD8DBFBC2E6FFD5DBFCC2E6FFEA
:100DC000D2DBFDC2E6FF54D3D9CFE6FFE1CFD9FF96
:100DD000A60E4D6E6F0E4E6E4F6A4DC0E6FFE66E6C
:100DE0004FC0E6FF7EEC37F0E552E552E552FE0ECD
:100DF000DBCFE6FF7DDFE5522F0EE66EB4DBFD0EA6
:100E0000DBCFE6FF75DFE5525D0EE66E31D3A3DB87
:100E100015E088DB13E08ADB11E08CDB0FE0AEC26B
:100E2000E6FF000E97DAAFC2E6FF010EA3DB020E6B
:100E300091DAB1C2E6FF030EAAEF09F0CCD28BDB48
:100E400023E070DB21E072DB1FE0500E0201AD5D9C
:100E500004E1200EEE6FB40E03D0240EEE6FB00E40
:100E6000EF6F1EDB71DBE2DA09E3EEDA07E325DB85
:100E700043DB7DDB030E0201EF2504D02F50301041
:100E800003E145DBAAEF09F0A6D265DB33E04ADBDC
:100E900031E04CDB2FE04EDB2DE0700E0201AD5D4A
:100EA00004E1B00EEE6F240E03D0B40EEE6F200EF0
:100EB000EF6F300E286EAEC229F0AFC22AF0B0C27A
:100EC0002BF0B1C22CF0B9DA0BE3C4DA09E3F5DA9E
:100ED000B1C2E6FF030E0201EE253CDA0DDB08D0BD
:100EE0002F50301007E113DB42DB030E0201EE2529
:100EF000AAEF09F070D20201AE51300812E2370EAB
:100F0000AE5D0FE20F0EAE15FF0F080DF350C00FD0
:100F1000EE6FAFC2E6FFE8502DDB0201EE29AAEF2B
:100F200009F0010EB56F1200310E0201AE5D01E253
:100F3000BFD0AE51390801E2BBD0AFC2E6FF73ECBF
:100F400037F0E552000901E1B3D0B0C2E6FF68EC2A
:100F500037F0E552000901E1ABD0BEDA500EAF5DCB
:100F60004CE12B0EB05D24E1AE51390A6CE0010A70
:100F70001DE00F0A19E0010A15E0030A11E0010A59
:100F80000DE0070A09E0010A05E0030A01E081D04B
:100F9000B7857FD0B7897DD0B8817BD0B78D79D028
:100FA000B88D77D0B88575D0B88973D0B78171D036
:100FB000AE51390A20E0010A1CE00F0A18E0010ACC
:100FC00014E0030A10E0010A0CE0070A08E0010A35
:100FD00004E0030A5EE1B7955CD0B7995AD0B891A6
:100FE00058D0B79D56D0B89D54D0B89552D0B89926
:100FF00050D0B7914ED0B9914CD02B0EB05D25E1B9
:10100000AE51390A20E0010A1CE00F0A18E0010A7B
:1010100014E0030A10E0010A0CE0070A08E0010AE4
:1010200004E0030A36E1B78734D0B78B32D0B883F7
:1010300030D0B78F2ED0B88F2CD0B8872AD0B88BAD
:1010400028D0B78326D0B98124D0AE51390A20E008
:10105000010A1CE00F0A18E0010A14E0030A10E07C
:10106000010A0CE0070A08E0010A04E0030A11E1A2
:10107000B7970FD0B79B0DD0B8930BD0B79F09D0BF
:10108000B89F07D0B89705D0B89B03D0B79301D0CD
:10109000B991B71DE66E150E5DD90201B81DE66E59
:1010A000160E58D90201B91DE66EFD0EAAEF09F021
:1010B00092D1EFD901E17AD035DA01E177D036DA91
:1010C00075E038DA73E0B2C2E6FF4CD96FE06C0E1F
:1010D0000201B35D03E0720EB35D68E16C0EB35DB7
:1010E00036E1300EAF5DF66FF76BF86BF96B100EF3
:1010F000446E270E456E466A476AF6C23FF0F7C255
:1011000040F0F8C241F0F9C242F07FEC3AF03BC047
:10111000F6F23CC0F7F23DC0F8F23EC0F9F2300EF4
:101120000201B05DC2D9E80E446E030E456E3DD992
:10113000300EB15DBAD9640E446E456A36D9300EB0
:10114000B25DB3D90A0E446E456A2FD904D0F66950
:10115000F769F869F969AD515D0A13E0060A09E01B
:10116000050A16E1500EAE5D02E1290E08D02D0EE3
:1011700006D0500EAE5D02E1A00E01D0A30EED6FC1
:1011800007D0500EAE5D02E1A60E01D0A90EED6FA4
:10119000F8C2E6FFED51DED8F7C2E6FF0201ED2905
:1011A000D9D8F6C2E6FF020EAFEF0AF014D171D91A
:1011B00053E0B8D951E0BAD94FE0BCD94DE0B2C242
:1011C000E6FFD0D849E0B3C2E6FFCCD845E0AFC2D5
:1011D00028F0B0C229F0B1C22AF0B2C22BF0B3C2DB
:1011E0002CF0C6EC36F02FC0F2F230C0F3F2020160
:1011F000F46BF56B100E446E0E0E456E466A476A30
:101200002FC03FF030C040F0F4C241F0F5C242F0D0
:101210007FEC3AF03BC0F2F23CC0F3F23DC0F4F296
:101220003EC0F5F2500E0201AE5D02E1170E01D094
:101230001B0EED6FF2C2E6FFE8508CD8F3C2E6FF5A
:101240000201ED2987D8F4C2E6FF020E88D9F5C263
:10125000E6FF030EAFEF0AF0BED0B5D804E24D5062
:10126000FC08000E4E540DE32DA003D002010D0E1C
:1012700002D002010C0EED6F2D50E66EED51AAEF7B
:1012800009F0A9D0A0D804E24D50FB08000E4E543E
:1012900005E32D50E66E140EAAEF09F09CD093D80A
:1012A00004E24D50FC08000E4E5405E32D50E66E4E
:1012B000900EAAEF09F08FD0300E2A6EAEC22BF03E
:1012C000AFC22CF079EC36F02D500F0805E32D500D
:1012D000E66E910EAAEF09F07ED0720E0201AE5DAD
:1012E0002EE1650E0201AF5D2AE1730E0201B05DD1
:1012F00026E1650E0201B15D22E1740E0201B25DCC
:101300001EE1F29EF29C040E0201F06FF16B0201ED
:10131000FF0ED880F055030EF1550FE3E668F0C2DA
:10132000E6FFF1C2E6FF0AEC3AF0E552E552E5527B
:101330000201F02B000EF123EAD7FF0003D00201D7
:10134000010EB56F1200E66EE66AB7EC3AF0E552B0
:10135000E5521200E66EE66A0AEC3AF0E552E55212
:10136000E55212004DEC37F0E552000912002FC093
:1013700051F030C052F0536A546A4D6A510E4E6EAD
:10138000250E4F6E020E506E4DC03FF04EC040F025
:101390004FC041F0426E2FC044F030C045F053C002
:1013A00046F054C047F029EF39F0466A476A7FECAF
:1013B0003AF03B500201F6273C50F7233D50F8230A
:1013C0003E50F9231200C0D879EC36F02D504D6E06
:1013D0004E6A4E3412000201010EB56F12004DC06C
:1013E00044F04EC045F04FC046F050C047F0E5EC29
:1013F0003AF03FC0DFF240C0E0F2120014C046F005
:101400004EC047F03FEC3BF041C00EF042C00FF041
:10141000010E1200F759000EF859000EF95912008A
:10142000F75B000EF85B000EF95B1200C6EC36F0BD
:10143000010E2F5C000E30581200C6EC36F0640E20
:101440002F5C000E30581200F40ED8802F54010E7D
:10145000305412000F0ED8802F54270E3054120033
:101460002FC04DF030C04EF0D8904E324D321200A9
:101470007AD8E552E7CFD9FF12000F0BF36EF00ECA
:1014800012000201B751000112000201B85100011F
:101490001200AEC2E6FF73EC37F0E552000912000D
:1014A000300E286E300E296E12003F6E406A416A7F
:1014B000426A120048DFFF081200AEC2E6FF0201D6
:1014C000EE5148DFAFC2E6FF0201EE2953D8020E0B
:1014D0000201EE25AAEF09F0150E35DFE81C020126
:1014E000B76F160E30DFE81C0201B86FFD0E2BDF60
:1014F000E81C0201B96F1200E6680201EF5137D80B
:101500000201EF2934D8020E0201EF251200E6682D
:101510000201EE512CD80201EE2929D8020E020157
:10152000EE251200AFC2E6FFB2EF09F0B0C2E6FF4F
:10153000B2EF09F0B1C2E6FFB2EF09F004DFE66EE8
:10154000120008DF00011200AEC22AF0AFC22BF079
:10155000B0C22CF01200AEC2E6FFB2EF09F00201F9
:10156000ED25AAEF09F008EC37F0E5521200F2DEA3
:0C157000E6681200EFDEB0C2E6FF1200D9
:04157C0061EC11F01D
:10158000FD0EDB5067E0FE0EDB5001E1C9D00E0A14
:101590005CE0030A55E0010A4EE0070A47E0010A51
:1015A00040E0030A39E0010A32E00F0A2BE0010AA9
:1015B00024E0030A1DE0010A16E0070A0FE0010A11
:1015C00008E0030A01E0ACD004017D0E376F040E81
:1015D000A5D004017F0E376F040EA0D00401810E48
:1015E000376F040E9BD004018B0E376F040E96D01C
:1015F00004018D0E376F040E91D00401B90E376FC0
:10160000030E8CD00401E70E376F000E87D0040163
:10161000E90E376F000E82D00401EF0E376F040E13
:101620007DD00401D70E376F030E78D00401F50E7C
:10163000376F030E73D00401830E376F040E6ED024
:101640000401380E376F050E69D004015B0E376F49
:10165000050E64D0FE0EDB5063E00E0A5BE0030A69
:1016600054E0010A4DE0070A46E0010A3FE0030AA0
:1016700038E0010A31E00F0A2AE0010A23E0030AF8
:101680001CE0010A15E0070A0EE0010A07E0030A60
:1016900047E10401590E376F040E40D004015B0E80
:1016A000376F040E3BD004015D0E376F040E36D049
:1016B0000401670E376F040E31D00401690E376FD5
:1016C000040E2CD00401AA0E376F030E27D004019C
:1016D000D80E376F000E22D00401DA0E376F000EDD
:1016E0001DD00401E00E376F040E18D00401C80E9F
:1016F000376F030E13D00401E60E376F030E0ED0C2
:1017000004015F0E376F040E09D00401290E376FF4
:10171000050E04D004015A0E376F050E386F03D042
:101720000401376B386B37C4F3FF38C4F4FF66EF3E
:1017300011F061EC11F0BBEC12F02D0802E1010E8A
:1017400001D0000E66EF11F0D0EC12F003E1F36A65
:10175000F46A38D00F0E39153C6F3D6BE80E3D032F
:10176000F3CF3DF4030E3C03F3503D27E80E3C035A
:10177000F3CF3CF4F4503D27FE0EDB50020FAFECEC
:1017800012F04D6E0F0E4D14640D3EEC12F0030F6F
:10179000AFEC12F04D6E0F0E4D140A0D3EEC12F030
:1017A000040FAFEC12F04D6E4E6A0F0E4D16000E88
:1017B0004E164D5004013C274E503D233CC4F3FFD0
:1017C0003DC4F4FF66EF11F0D0EC12F002E1010E1F
:1017D00023D00F0E3915640DF3503A6F3B6BFE0E9C
:1017E000DB50020FAFEC12F00F0B0A0DF3504D6EF1
:1017F0004E6AF35004013A274E503B23FE0EDB5055
:10180000030FAFEC12F00F0B4D6E4E6AE85004015F
:101810003A274E503B233A5166EF11F061EC11F03C
:10182000BBEC12F064EC12F002E0395101D0000E72
:1018300066EF11F061EC11F0FA0EDBCFE6FF46EC3B
:1018400011F0E66E87EC11F0E552E750EF6E87EC91
:1018500011F0EF500F0B00091AE087EC11F0EF5078
:10186000800B01E0010EE66E87EC11F0EF500F0BDC
:10187000E66E84DEE552E552F3CF4DF0F4CF4EF044
:10188000FD0EDBCFE9FFFE0E56EC12F008D091EC16
:1018900012F0F80EDBCFEEFFF90EDBCFEDFFF50E09
:1018A000DBCFE6FF51DFE552F3CF4DF0F4CF4EF042
:1018B000F60EDBCFE9FFF70E56EC12F0F50EB2ECA8
:1018C00012F0EF0EEF14F310EF6EF20EDBCFE6FF27
:1018D0007BDFE552E66EF30EDBCFE9FFF40EDBCFE4
:1018E000EAFFE552E750EF6EF20EB2EC12F0F3466B
:1018F000DF0EEF14F310EF6EEF0EDBCFE6FF8EDF9F
:10190000E552E66EF00EDBCFE9FFF10EDBCFEAFF2A
:10191000E552E750EF6E66EF11F061EC11F0020E48
:10192000E126BBEC12F0DF6EFE0EDB28AFEC12F00E
:10193000E76E010EE7CFDBFFFF0EDF5C06E1010E75
:10194000DB50FF0802E1DE6ADD6ADECF4DF0DDCF5D
:101950004EF04DC0F3FF4EC0F4FF020EE15C02E218
:10196000E16AE552E16E66EF11F0010EC26EC16AE6
:10197000960EC06E0F010F0E5D6F050E5C6F336A21
:10198000080EAFEC12F0FF0809E1E66A080EE66EF9
:10199000E66A0AEC3AF0E552E552E552080EAFEC81
:1019A00012F00401006F3B0EE66E250EE66E040E8B
:1019B000E66E360EE66E130EE66E040EE66E300E22
:1019C000E66E190EE66E040EE66E0A0EE66E050E63
:1019D000E66E3D0EE66E010EE66E040EE66E070E36
:1019E000E66E040E7FEC11F04B0EE66E260EE66EF0
:1019F000040EE66E460EE66E140EE66E040EE66EFD
:101A0000400EE66E1B0EE66E040EE66E0C0EE66EE3
:101A1000050EE66E4D0EE66E020EE66E040EE66EE6
:101A2000090EE66E040E7FEC11F05B0EE66E270EDB
:101A3000E66E040EE66E560EE66E150EE66E040EAB
:101A4000E66E500EE66E1D0EE66E040EE66E190E84
:101A5000E66E050EE66E5D0EE66E030EE66E040E95
:101A6000E66E0B0EE66E040E7FEC11F06B0EE66E6A
:101A7000280EE66E040EE66E660EE66E160EE66E36
:101A8000040EE66E600EE66E1F0EE66E040EE66E47
:101A90001B0EE66E050EE66E6D0EE66E040EE66E2D
:101AA000040EE66E0D0EE66E040E7FEC11F07B0E5A
:101AB000E66E290EE66E040EE66E760EE66E170EE4
:101AC000E66E040EE66E700EE66E210EE66E040EF5
:101AD000E66EDE0EE66E040EE66E7D0EE66E050E1A
:101AE000E66E040EE66E0F0EE66E040E7FEC11F04D
:101AF0008B0EE66E2A0EE66E040EE66E860EE66E1F
:101B0000180EE66E040EE66E800EE66E230EE66E8E
:101B1000040EE66EED0EE66E040EE66E8D0EE66EBB
:101B2000060EE66E040EE66E110EE66E040EE7DBA0
:101B3000C00ECEEC11F0F3CF42F4F4CF43F4C80E54
:101B4000CEEC11F0F3CF44F4F4CF45F4D00ECEEC4C
:101B500011F0F3CF46F4F4CF47F4D80ECEEC11F0E9
:101B6000F3CF48F4F4CF49F4E00ECEEC11F0F3CF0C
:101B70004AF4F4CF4BF4E80ECEEC11F0F3CF4CF472
:101B8000F4CF4DF412009DDBFB0EDBB8E4DBC1ECBF
:101B900011F03FC03EF440C03FF4FB0EDB500008A4
:101BA0000AE2FB0EDB500F0B040105E0D8903F3337
:101BB0003E33E806FBE1335025E0020A10E0030A59
:101BC00021E1E1EC11F004013E514D5C3F514E58D2
:101BD00016E2A4DB41503E5F42503F5B19D0E1EC7E
:101BE00011F004014D503E5D4E503F5908E296DB26
:101BF0003E51415C3E6F3F5142583F6F09D03E6BB2
:101C00003F6B06D08BDB415004013E2742503F23FF
:101C10003EC4F3FF3FC4F4FF59D353DBFB0EDBB8E4
:101C20009ADBAFDB3FC040F440C041F4FB0EDB5019
:101C300000080AE2FB0EDB500F0B040105E0D89010
:101C400041334033E806FBE1335031E0020A18E04B
:101C5000030A2DE1FC0E040140254D6E7F0E41214B
:101C60004E6EFD0EDBCF4FF0FE0EDBCF50F069EC79
:101C700012F018E253DB4150405F4250415B1DD0EF
:101C8000A0DBFC0E4D267F0E4E2204014D50405D20
:101C90004E50415907E242DB4051415C406F415197
:101CA000425803D0040E406F800E416F06D036DBE1
:101CB0004150040140274250412340C4F3FF41C436
:101CC000F4FF04D3FEDAE150FB0FC0EC12F0FC0E7F
:101CD000D880EE54FF0EED5403E2FC0EC9DBDB6846
:101CE0004ADB01E0F7DAF2D2ECDA72DB4E340FE2D3
:101CF0004D50FC087F0E4E540AE2FC0EF36EFB0EB4
:101D0000F3CFDBFF7F0EF36EFC0EF3CFDBFF33DB95
:101D100001E0E0DADBD2D5DA5BDBD8804E5004E7B5
:101D2000840E4D5CFF0E4E5804E2840EA1DBDB688E
:101D30000BD04EDB4E3408E24D507C08000E4E5462
:101D400003E27C0E95DBDB6A16DB05E091EC12F01A
:101D5000FB0EDBCFEFFFBAD2A5EC12F0000A1AE0BF
:101D60000C0A14E0060A10E00F0A0CE00E0A08E064
:101D70000A0A04E0020A60E1020E24D0040E22D016
:101D8000080E20D0100E1ED0400E1CD0020EDB6AB2
:101D9000020E0AD0FE0EDB0404E0FE0EDB50030848
:101DA00008E1020EDB6A080EF36E030EF3CFDBFFD1
:101DB0000AD0FE0EDB50050804E0FE0EDB500608DC
:101DC0003BE1200E7ADB75DA800B01E0010E010B9E
:101DD00004E07C0EDE6E040E03D0580EDE6E040EA0
:101DE0005DDB2AE066DA0F0B03080BE062DA0F0B0B
:101DF00000090BE1FE0EDB0404E0FE0EDB500308DD
:101E000004E14ADA66DB03E30DD0BFDB0BE2020E2E
:101E1000DBCF4DF0030EDBCF4EF0E1DAEE124E5089
:101E2000ED120AD0020EDB1C4D6E030EDB1C4E6E53
:101E3000D6DAEE164E50ED16040EE15C02E2E16ACF
:101E4000E552E16E43D281DB070A04E00F0A28E184
:101E5000020E01D0040E31DB2CDA800B01E0010E02
:101E6000010B04E0E50EDE6E000E03D0D60EDE6E32
:101E7000000E14DB15E01DDA0F0B080804E10CDA84
:101E800028DB03E307D081DB05E2B3DA020EDB5087
:101E9000EF1206D0020EDB1C4D6EABDA4D50EF1682
:101EA000040EE15C02E2E16AE552E16E0FD209DA6A
:101EB000E150F80F65DBEE50ED1006E036DA4CDF4E
:101EC0006ADB33DAC0DF67DB01D2FBD900C44DF037
:101ED0004E6A4DBE4E684D50C3264E50C422C4506B
:101EE000F00B02E0C36AC46A010E0F0B05E0D89044
:101EF000C432C332E806FBE1FE0EDB50050804E005
:101F0000FE0EDB5006080BE1C3CF4DF0C4CF4EF000
:101F1000D8904E324D324D50C3264E50C422FE0E44
:101F2000DB50060A01E138D1030A01E1FBD0010AC6
:101F300001E1BAD0070A01E17DD0010A3DE0030AC0
:101F400001E063D1040101512EDA31E201AB02D08C
:101F5000020E03D001A903D0010E336E01D0336A03
:101F600001510F0B0D0814E001510F0B0E0810E08A
:101F700049DAE3DA42C4E6FF43C4E6FF19DA010EA8
:101F8000E66E040EE66E010E7CD9A8DA9BDE0ED05A
:101F900039DAD7DA040101510F0B0D0804E1BCDA7C
:101FA0009DDAA2DE03D0B8DA99DAB5DEC1DAC3CFA2
:101FB0002CF4C4CF2BF429D104010251F4D935E219
:101FC00002AB02D0020E03D002A903D0010E336E81
:101FD00001D0336A02510F0B0D0818E002510F0BAC
:101FE0000E0814E002510F0B000910E014DAA5DA14
:101FF00044C4E6FF45C4E6FFDBD9020EE66E040EDC
:10200000E66E020E3ED96FDA5DDE0ED004DA99DAA2
:10201000040102510F0B0D0804E17EDA64DA64DE7C
:1020200003D07ADA60DA77DE83DAC3CF2EF4C4CF56
:102030002DF4EBD004010351B6D931E203AB02D049
:10204000020E03D003A903D0010E336E01D0336A10
:1020500003510F0B0D0814E003510F0B0E0810E095
:10206000E3D96BDA46C4E6FF47C4E6FFA1D9030E05
:10207000E66E040EE66E030E04D93ADA23DE0ED0C5
:10208000D3D95FDA040103510F0B0D0804E144DAE0
:102090002FDA2ADE03D040DA2BDA3DDE49DAC3CF6D
:1020A00030F4C4CF2FF4B1D0040104517CD935E20F
:1020B00004AB02D0020E03D004A903D0010E336E8C
:1020C00001D0336A04510F0B0D0818E004510F0BB7
:1020D0000E0814E004510F0B000910E0AED92DDA00
:1020E00048C4E6FF49C4E6FF63D9040EE66E040E59
:1020F000E66E040EC6D801DAE5DD0ED09ED921DAEF
:10210000040104510F0B0D0804E106DAF6D9ECDDE9
:1021100003D002DAF2D9FFDD0BDAC3CF32F4C4CF39
:1021200031F473D0040105513ED931E205AB02D040
:10213000020E03D005A903D0010E336E01D0336A1D
:1021400005510F0B0D0814E005510F0B0E0810E0A0
:102150007DD9F3D94AC4E6FF4BC4E6FF29D9050E61
:10216000E66E040EE66E050E8CD8CCD9ABDD0ED033
:102170006DD9E7D9040105510F0B0D0804E1CCD945
:10218000C1D9B2DD03D0C8D9BDD9C5DDD1D9C3CF3E
:1021900034F4C4CF33F439D00401065104D931E208
:1021A00006AB02D0020E03D006A903D0010E336E97
:1021B00001D0336A06510F0B0D0814E006510F0BC6
:1021C0000E0810E04CD9B9D94CC4E6FF4DC4E6FF67
:1021D000EFD8060EE66E040EE66E060E52D897D9BC
:1021E00071DD0ED03CD9ADD9040106510F0B0D089D
:1021F00004E192D98CD978DD03D08ED988D98BDDD2
:1022000097D9C3CF36F4C4CF35F460D008500A0A4A
:1022100029E0030A23E0010A1DE00F0A17E0010A82
:1022200011E0030A0DE0010A07E0070A13E0010AC2
:102230000DE0030A1EE106D0040EBFD8A30E15D090
:10224000050E11D0010EB9D88B0E0FD0020EB5D8E5
:10225000870E0BD0030EB1D8830E07D0040EADD875
:10226000AB0E03D0060EA9D88F0EE66E55EC3BF0F0
:10227000E5521FEF3CF05CD9F3CF34F0F4CF35F0EA
:102280001200E66E14DE87D98CEF12F0E66AB7EC26
:102290003AF0E552E5521200FA0EDBCF4DF0FB0E9C
:1022A000DBCF4EF0F80EDBCF4FF0F90EDBCF50F066
:1022B0001200FC0EDBCFE9FFFD0EDBCFEAFFEF5093
:1022C0001200D9CFE6FFE1CFD9FF1200E552E7CFE8
:1022D000D9FF120026D9FB0EDBCFEFFFFB0EFC0E61
:1022E000DBCF4EF04EC04DF04E6A010EE76E19D9AD
:1022F000E750E926000EEA224DC0EFFF1200E66E1D
:102300001AEC0CF04D6E100EE15E4D501200FB0EFB
:10231000DBCFE9FFFC0EDBCFEAFF1200FD0EDBCFC7
:1023200041F0FE0EDBCF42F01200F80EDBCFE6FFED
:10233000F90EDBCFE6FFFA0EDBCFE6FFFB0EDBCFBD
:10234000E6FFFC0EDBCFE6FFFD0EDBCFE6FFFE0E69
:10235000DBCFE6FF1200FB0EDB98D950FD0F10D942
:102360000A0EEC02F3CFEDFF0A0EEF02F3CFEEFF01
:10237000F450ED261200D950FD0F02D9EE50ED10A9
:102380001200FC0EDB504D6E4E6A416E4EC042F0A4
:10239000C3CF46F0C4CF47F05DEF39F0E66E8DEC69
:1023A0000CF0E55212000F0B4D6E0F0E4D5C12003B
:1023B000F3CFE6FFF4CFE6FF1200E66E86DDE552CE
:1023C0001200FD0EDBCF4DF0FE0EDBCF4EF0120003
:1023D000FB0EDBCF4DF0FC0EDBCF4EF01200DECF5C
:1023E000E9FFDDCFEAFF140EE926000EEA224D5088
:1023F0001200DECFE9FFDDCFEAFF060EE926000E70
:10240000EA22120025C4E6FF13C4E6FF19C4E6FF62
:102410001AC4E6FF120026C4E6FF14C4E6FF1BC47C
:10242000E6FF1CC4E6FF120027C4E6FF15C4E6FF62
:102430001DC4E6FF1EC4E6FF120028C4E6FF16C452
:10244000E6FF1FC4E6FF20C4E6FF120029C4E6FF32
:1024500017C4E6FF21C4E6FF22C4E6FF12002AC427
:10246000E6FF18C4E6FF23C4E6FF24C4E6FF12001B
:10247000F36EFB0EF3CFDBFFFC0E1200F3500401F2
:102480003C27F4503D23FE0EDB5012004D50010B53
:10249000F36EF346F346F346F3461200DD6ED9CFF2
:1024A000E9FFDACFEAFFEE50ED101200DBCFEAFFD2
:1024B000F3CFEEFF4EC0EDFF1200F36E020EF3CF2E
:1024C000DBFF030EDB6A12000401396FFF0E395D7A
:1024D00012004D504F5C4E505058120007C4E6FF9A
:1024E00008C4E6FF120009C4E6FF0AC4E6FF1200B2
:1024F0000BC4E6FF0CC4E6FF12000DC4E6FF0EC4D9
:10250000E6FF12000FC4E6FF10C4E6FF120011C47C
:10251000E6FF12C4E6FF120034C0E6FF35C0E6FF56
:102520001200FD0EDBCFE9FFFE0EDBCFEAFF12004B
:10253000E552E552E552E5521200C3EC0DF03BEFD7
:1025400011F00DEC0EF03BEF11F0BBDE040EE126B6
:10255000020EDB6A030EDB6AACDE0F0B1200E66EC6
:1025600046EF11F0DBCFE6FF99EC0BF0E5524D6E34
:10257000CEDE46EF12F0FE0EDBCFE6FF46EF11F0A7
:10258000E96EFF0EDA20EA6E120086DE4F504D5CD7
:1025900050504E5812004D6E070EE15E4D50120025
:0C25A00090DEFE0EDB28DBDF64EF12F0A3
:0425AC00376A386AE8
:1025B00012009E0E4D6E710ED1EF19F09B0E4D6EF6
:1025C000710ED1EF19F0910E4D6E710ED1EF19F021
:1025D0008C0E4D6E710ED1EF19F0870E4D6E710E8F
:1025E000D1EF19F01BEC1AF0FE0EDB5004E0810E67
:1025F0004D6E710E03D07B0E4D6E710ED1EC19F045
:1026000020EF1AF0D9CFE6FFE1CFD9FFFE0EDB288D
:10261000E66EE66AB7EC3AF0E552E5520001FA6F71
:10262000FAC026F0FAC027F00001263A0F0E26164F
:102630002650090802E2070E2626300E26260F0E27
:1026400027162750090802E2070E2726300E2726F4
:102650002650E66E08EC37F0E5522750E66E08EC9F
:1026600037F0E552FE0EDBCFE6FFE66AB7EC3AF054
:10267000E552E5520001FA6FFAC026F0FAC027F0E1
:102680000001263A0F0E26162650090802E2070E10
:102690002626300E26260F0E27162750090802E29E
:1026A000070E2726300E27262650E66E08EC37F058
:1026B000E5522750E66E08EC37F0E552E552E7CFD9
:1026C000D9FF12001BEC1AF05B0EDBEC19F0050EC3
:1026D000E66EFE0E7BEC1AF0040EE66EFD0E7BEC51
:1026E0001AF0FC0EDBCFE6FFE66A86EC1AF000017A
:1026F000F26FFF0EF25D01E1F26B300EF225DBECC2
:1027000019F05D0E67EC1AF020EF1AF01BEC1AF0CE
:10271000E15010EC1AF00F0B000924E1FE0EDB5023
:10272000060A1BE0030A17E0010A10E0070A09E0A5
:10273000010A05E0030A01E07AD04ADF03D048DF4E
:1027400006D04BDF6E0E4D6E710E6FD046DF610E00
:102750004D6E710E6AD03CDF01D03FDF540E4D6EDE
:10276000710E63D0D95010EC1AF0800B02E035DF07
:1027700001D02EDFD95010EC1AF00F0B0E0A4EE0EC
:10278000030A48E0010A42E0070A3CE0010A36E099
:10279000030A30E0010A2AE00F0A24E0010A1EE0E1
:1027A000030A18E0010A12E0070A0CE0010A06E039
:1027B000030A38E1470E4D6E710E37D03A0E4D6E5A
:1027C000710E33D02D0E4D6E710E2FD0200E4D6E2A
:1027D000710E2BD0130E4D6E710E27D0060E4D6E5E
:1027E000710E23D0F90E4D6E700E1FD0EC0E4D6E93
:1027F000700E1BD0DF0E4D6E700E17D0D20E4D6EC8
:10280000700E13D0C50E4D6E700E0FD0B80E4D6EFB
:10281000700E0BD0AB0E4D6E700E07D09E0E4D6E2F
:10282000700E03D0910E4D6E700ED1EC19F020EFAA
:102830001AF0C4DEC3DE8A0E4D6E700ED1EC19F0B4
:10284000330EDBEC19F02E0EDBEC19F0350EDBEC61
:1028500019F0300E67EC1AF0230EDBEC19F0000EC5
:10286000A9EC1AF0010EA9EC1AF0020EA9EC1AF06C
:10287000030EE5EC19F067EC1AF05B0EDBEC19F0D7
:10288000140E8BEC1AF02C0EDBEC19F00C0E8BEC0A
:102890001AF02F0EDBEC19F00D0E8BEC1AF05D0E1A
:1028A00067EC1AF00401003508E32D0EDBEC19F09B
:1028B0000401001D010FE66E05D02B0EDBEC19F0B4
:1028C00000C4E6FF0FEC37F0E552150EE5EC19F009
:1028D000E81C0001ED6F160EE5EC19F0E81C000194
:1028E000EE6FFD0EE5EC19F0E81C0001EF6F66DEFF
:1028F0006ADE7B0E4D6E700E71EC1AF0040B01E077
:10290000010EA3EC1AF0080B01E0010EE9EC19F03E
:10291000740E4D6E700ED1EC19F0030EE66E200EA3
:1029200081EC1AF0030EE66E240E6BEC1AF0650EC5
:102930004D6E700E71EC1AF0100B01E0010EA3EC5D
:102940001AF0200B01E0010EE9EC19F05E0E4D6E5D
:10295000700ED1EC19F0040EE66EB00E81EC1AF098
:10296000040EE66EB40E6BEC1AF04F0E4D6E700E48
:1029700074EC1AF0010BA6EC1AF0020B01E0010E48
:10298000E9EC19F02D0EE66E290E00EC1AF0400E5F
:102990004D6E700E71EC1AF0400B01E0010EA3ECCD
:1029A0001AF0800B01E0010E8EEC1AF0310E4D6E24
:1029B000700E74EC1AF0400B01E0010EA6EC1AF058
:1029C000800B01E0010E8EEC1AF0220E4D6E700E9F
:1029D00074EC1AF0040B01E0010EA6EC1AF0080BDF
:1029E00001E0010EE9EC19F0A30EE66EA00E00EC7A
:1029F0001AF0130E4D6E700E74EC1AF0100B01E00D
:102A0000010EA6EC1AF0200B01E0010EE9EC19F022
:102A1000A90EE66EA60E00EC1AF0040E4D6E700EB6
:102A200071EC1AF0010BA3EC1AF0020B01E0010E9D
:102A30008EEC1AF0EE0E4D6E6F0ED1EC19F0000117
:102A4000EF51010BE9EC19F00A0EE5EC19F0E81C66
:102A50000001F36FB3DDE70E4D6E6F0ED1EC19F090
:102A60003D0E64EC1AF0010EF2EC19F03B0EE66E2E
:102A7000360EE66E300EEEEC19F0C00EF8EC19F0E2
:102A8000080E77EC1AF0E00E4D6E6F0ED1EC19F0D7
:102A90004D0E64EC1AF0020EF2EC19F04B0EE66EDD
:102AA000460EE66E400EEEEC19F0C80EF8EC19F08A
:102AB000040E77EC1AF0D90E4D6E6F0ED1EC19F0B2
:102AC0005D0E64EC1AF0030EF2EC19F05B0EE66E8C
:102AD000560EE66E500EEEEC19F0D00EF8EC19F032
:102AE000020E77EC1AF0D20E4D6E6F0ED1EC19F08B
:102AF0006D0E64EC1AF0040EF2EC19F06B0EE66E3B
:102B0000660EE66E600EEEEC19F0D80EF8EC19F0D9
:102B1000010E77EC1AF0CB0E4D6E6F0ED1EC19F062
:102B20007D0E64EC1AF0050EF2EC19F07B0EE66EE9
:102B3000760EE66E700EEEEC19F0E00E91EC1AF0E7
:102B4000C40E4D6E6F0ED1EC19F08D0E64EC1AF0C0
:102B5000060EF2EC19F08B0EE66E860EE66E800E17
:102B6000EEEC19F0E80E91EC1AF028DDDEEF12F031
:102B7000310E0201AE5D01E2B8D00201AE5136085D
:102B800001E2B3D0730E0201AF5D01E0AED0740E6E
:102B90000201B05D01E0A9D06E0E0201B15D01E05D
:102BA000A4D03A0E0201B25D01E09FD0C00EF21433
:102BB0000001FD6F3F0EF2168B8A8B88C00E4D6EA2
:102BC0006F0E4E6E4F6A4DC0E6FF4EC0E6FF4FC01F
:102BD000E6FF7EEC37F0E552E552E552AEC2E6FF85
:102BE00008EC37F0E5523F0EE66E08EC37F0E552A0
:102BF0000001F96B400E0001F95D17E29EBA02D0A8
:102C00000400FCD7AECFF7F00001F951EA6A960F45
:102C1000E96E040EEA22F7C0EFFF0D0E0001F75D2A
:102C200001E103D00001F92BE5D70201AE51360ACC
:102C300028E0030A20E0010A18E0070A11E0010A6F
:102C400009E0030A01E023D00001800EFB6F020EB1
:102C5000FC6F1ED00001C00EFB6F020EFC6F18D07F
:102C60000001FB6B030EFC6F13D00001400EFB6FE5
:102C7000030EFC6F0DD00001800EFB6F030EFC6F86
:102C800007D00001C00EFB6F030EFC6F01D000D017
:102C90000001FA6B0001F9510001D880FA5519E3DF
:102CA0000001FA51EA6A960FE96E040EEA22EF502B
:102CB000E66EFBC0E6FFFCC0E6FF0AEC3AF0E55228
:102CC000E552E5520001FB2B000EFC230001FA2B1C
:102CD000E1D700017A89258025928B9A8B98AECF17
:102CE000F7F00001FD51F21203D00201010EB56FA1
:102CF0001200CEDB01E27ED0AE51360801E27AD07E
:102D0000AFC2E6FF73EC37F0E552000973E0B0C2E2
:102D1000E6FF59EC37F0E55200096CE0B0C2E6FF7F
:102D2000300EE66E2DEC36F0E552E55200010F0B49
:102D3000F36EF00EF015F310F06F500E0201AF5D60
:102D400002E1000E01D0010E0001F09FE8B0F08F0B
:102D50000201AE51360A19E0030A14E0010A0FE03D
:102D6000070A0AE0010A05E0030A12E100013D0E2C
:102D70000ED000014D0E0BD000015D0E08D00001F9
:102D80006D0E05D000017D0E02D000018D0EF46F96
:102D90000001F4511ADB0001F16FF0C0E6FFF451BD
:102DA0000FDB0001F1510F0B0B0A13E0010A0AE0DF
:102DB0000C0A01E01200F151800B02E02D0E0FD041
:102DC000290E0DD0F151800B02E0A30E08D0A00E09
:102DD00006D0F151800B02E0A90E01D0A60EF46FCF
:102DE000E668E850EDDAE6680001F429E9DAE66819
:102DF000020EA5D311D34CDB3AE3AE51360837E3CC
:102E000016DB35E0B0C2E6FFF6DA31E0B1C2E6FF2C
:102E1000F2DA2DE0B2C2E6FFEEDA29E0B3C2E6FF55
:102E2000EADA25E00201AE51360A19E0030A14E09D
:102E3000010A0FE0070A0AE0010A05E0030A12E1AD
:102E40000001300E0ED00001400E0BD00001500EDC
:102E500008D00001600E05D00001700E02D0000104
:102E6000800EF46F19DBB3C2E6FF040E68D3D4D230
:102E70000FDB33E3AE51360830E3D9DA2EE0B0C2CF
:102E8000E6FFB9DA2AE0B1C2E6FFB5DA26E0B2C25F
:102E9000E6FFB1DA22E00201AE51360A19E0030A78
:102EA00014E0010A0FE0070A0AE0010A05E0030A3C
:102EB00012E10001360E0ED00001460E0BD00001CB
:102EC000560E08D00001660E05D00001760E02D025
:102ED0000001860EF46F4CEF1AF09ED2D9DA39E376
:102EE000AE51340836E3A3DA34E00A0E6EDA00019C
:102EF000F36F2B0E0201AF5D15E1AE51340A0FE006
:102F0000070A0AE0010A05E0030A1EE10001F3973F
:102F10001BD00001F39518D00001F39315D00001E8
:102F2000F39112D0AE51340A0CE0070A08E0010A0E
:102F300004E0030A09E1F80E05D0F40E03D0F20E06
:102F400001D0F10E0001F313F3C0E6FF0A0EE0EF2B
:102F500019F062D29DDA3AE3AE51360837E38CDAE3
:102F600035E0B0C2E6FFE2DA31E0300E0201AF5DDB
:102F70000001F26F2B0E0201B05D02E10001F28947
:102F80000201AE51360A19E0030A14E0010A0FE00B
:102F9000070A0AE0010A05E0030A12E100013B0EFC
:102FA0000ED000014B0E0BD000015B0E08D00001CB
:102FB0006B0E05D000017B0E02D000018B0EF46F6A
:102FC000F2C0E6FF0001F451E0EF19F025D2AEC2E5
:102FD000E6FFACDA1BE050DA19E0AFC2F3F0410EC5
:102FE0000001F35D02E3070EF35F300EF35F2D0E79
:102FF0000201AE5D04E10001F31DF36FF32BF3C09A
:1030000000F4F3C0E6FF080EE0EF19F005D213DA82
:10301000410ED1D9FE0EDBCFE6FF08EC37F0E552CA
:103020003D0EC9D90001F96B400EF95D1CE2FC0EA2
:10303000DBCFE6FFFD0EDBCFE6FF68DA0001F86FBD
:10304000FC0EDB2AFD0E01E3DB2AFF0EF85D0BE030
:103050000D0EF85D08E0F8C0E6FF08EC37F0E55229
:103060000001F92BE1D70D0EA6D90A0EA4D9E8D19B
:103070000201B56B375001E0D3D03750EA6AAD0F8B
:10308000E96E020EEA2236C0EFFF36502A0A01E14D
:10309000BBD0690A01E1B8D0140A01E1B5D0080A31
:1030A00001E1B2D0110A01E1ABD00A0A01E1A8D0D6
:1030B000140A01E1A5D0030A01E1A2D0020A01E14C
:1030C0009FD00B0A01E19CD0260A01E199D03D0A6C
:1030D00001E196D0670A01E193D0050A01E18CD0A5
:1030E000530A01E189D0030A01E186D02A0A01E1ED
:1030F0007FD0270A01E17CD0130A01E179D0350A9B
:1031000073E00A0A71E00C0A6FE0050A6DE0060A36
:103110006BE0620A61E05F0A0AE05E0A06E0020A0A
:1031200001E076D0328E31987AD0FF0078D00D0E43
:10313000E66E08EC37F0E5520A0EE66E08EC37F062
:10314000E552F29E800EE66E020EE66E310EE66EDF
:103150005EDFE552E552E552C00EE66E020EE66E07
:10316000320EE66E54DFE552E552E552E66A030E92
:10317000E66E330EE66E4BDFE552E552E552400E49
:10318000E66E030EE66E340EE66E41DFE552E55262
:10319000E552800EE66E030EE66E350EE66E37DF04
:1031A000E552E552E552C00EE66E030EE66E360EAF
:1031B000E66E2DDFE552E552E5520D0EE66E08ECA7
:1031C00037F0E5520A0EE66E08EC37F0E552719ED4
:1031D000719CF28E319823D0F29E19EC14F0719EFE
:1031E000719CF28E31981BD0060E386E372A17D09C
:1031F000050E386E372A13D0040E386E372A0FD0DA
:10320000030E386E372A0BD0020E386E372A07D0DD
:103210000201010EB56F386A376A319800D08CD040
:103220003850375C0AE23750EA6AAD0FE96E020E99
:10323000EA2236C0EFFF372A7FD03750080801E274
:1032400078D03750EA6AAD0FE96E020EEA2236C036
:10325000EFFF0201AD515F0A5FE0790A5AE0710A9F
:1032600057E0290A52E0020A4DE0110A49E0470AF4
:1032700045E0700A41E0190A3DE01A0A39E0010A06
:1032800035E01C0A31E0150A2CE0030A27E00C0A9D
:1032900022E0050A20E0060A1EE0130A19E00F0AE0
:1032A00014E0310A0FE0030A0DE0230A08E0030AE4
:1032B00006E0700A01E033D007EC07F034D01FECD1
:1032C00007F031D045EC07F02ED07BEC07F02BD087
:1032D00094EC07F028D059EC08F025D0D7EC08F092
:1032E00022D02DEC09F01FD004DD1DD084DD1BD0D1
:1032F000BFDD19D0F3DD17D02DDE15D068DE13D079
:1033000037DC11D042EC09F00ED06DEC09F00BD097
:103310000AD04FEC09F007D05CEC09F004D00201B0
:10332000010EB56F00D037C0F6F0376A386A3198B1
:1033300003D0386A376A31980201B55131E0AD0ED9
:103340004D6E6F0E4E6E4F6A4DC0E6FF4EC0E6FFEB
:103350004FC0E6FF7EEC37F0E552E552E552000142
:10336000F56B0001F6510001D880F5550FE300011F
:10337000F551EA6AAD0FE96E020EEA22EF50E66EF1
:1033800008EC37F0E5520001F52BEBD70D0EE66E99
:1033900008EC37F0E5520A0EE66E08EC37F0E5521D
:1033A00012004E6E4F6A4DC0E6FFE66E4FC0E6FF5C
:1033B0007EEC37F0C0D0E66E08EC37F0E552120034
:1033C000E66EE66A0AEC3AF0B6D0E66EE66A86EF9A
:1033D0001AF0E66EF2EC12F0E5521200E66E62ECC4
:1033E00013F0A9D0E66E86EC13F0E552E552120018
:1033F00098D8D9EF12F04DEC37F0E55200091200E1
:10340000E66EE4EC06F0E552E552E3EF12F02DEC47
:1034100037F0E552E55212000201010EB56F1200BD
:10342000FD0FE96EFF0EDA20EA6EEF501200AFC218
:10343000E6FF96EF1AF0D9CFE6FFE1CFD9FF1200F1
:10344000E552E7CFD9FF1200E8EC12F00001ED5190
:103450001200EDEC12F00001ED511200E8EC12F058
:103460000001EE511200EDEC12F00001EE511200DD
:103470000001F06FE66E1200AFC2E6FF59EC37F0C4
:10348000E55200091200E66E23EC37F0E552120017
:10349000310E0201AE5D1200AFC2E6FF0001F45131
:1034A0008FDFB0C2E6FF0001F4298ADFB1C2E6FF78
:1034B000020E0001F42584DFB2C2E6FF030E3FD006
:1034C00088DF2F0EDBEF19F080DF38EF1AF073DFA3
:1034D000200EDBEF19F0E66E9ADF5D0E6CDFE3EF96
:1034E00012F05FDF24EF1AF05CDF2EEF1AF000011C
:1034F000F315E9EF19F0DBCFE6FF89DF2C0EDBEFE8
:1035000019F0E66E84DF2F0EDBEF19F0B7EC3AF01E
:10351000E552E552120059DF43EF1AF05ADFE3EFAC
:1035200012F0E66E02EC13F0E552120068EC37F090
:10353000E55200091200E552E552E5521200000181
:10354000F425E0EF19F0BCDF29EF1AF0B9DF33EF13
:083550001AF03BDFDBEF19F07C
:08355800100E0101121905E13A
:10356000FE0E131902E1010E141901E180D0140EB0
:10357000121905E1F20E131902E1010E141973E09C
:10358000110E121905E1F20E131902E1010E1419C0
:1035900062E0050E121905E1F20E131902E1010EA7
:1035A000141955E0010E121905E1F20E131902E18A
:1035B000010E141948E0125105E1F20E131902E14F
:1035C000010E14193CE00D0E121905E1F10E13194C
:1035D00002E1010E14192FE0140E121905E1F00E8C
:1035E000131902E1010E141923E0125105E1EE0E48
:1035F000131902E1010E141916E012513BE1EE0E0F
:10360000131938E1145136E125B44DD0FF0E0101F4
:103610001A5D06E00001695101011A5D44E125923D
:1036200000017A89120000017A8D0FC1B8F11200F1
:1036300000017B85120000017C877C89120000015B
:103640007D857D87120000017D897D8B1200000140
:103650007D8D7D8F120000017E857E877E897E8B29
:103660007E8D7E8F120000017F837F851200000116
:10367000878112000001695101011A5D03E0FF0E0C
:103680001A5D11E10FC103F10101010E076F086915
:1036900009690A690B6912C10CF113C10DF114C15A
:1036A0000EF100017A811200D9CFE6FFE1CFD9FFF8
:1036B0000101FA6BFC0EDB50FA5D74E27AEC21F04A
:1036C000B2EC21F0E552E750EF6EE9EC21F001E3B6
:1036D000DB2AFA51B2EC21F0EF500A0A5DE0030A4E
:1036E00056E0010A50E00F0A4AE0010A55E0030AD9
:1036F00041E0010A3AE0070A34E0010A0AE0030A5D
:103700004BE1E9EC21F001E3DB2AE9EC21F044E3B1
:1037100026D0010EE76E05EC22F0E750E926000EF8
:10372000EA22EFCF4FF04FC050F04F6A05EC22F085
:10373000EF5000014F104D6E50C04EF00101FA5194
:1037400029EC21F04DC0EEFF4EC0EDFFFA5129ECFF
:1037500021F0EE52070EED16E9EC21F01DE3DB2A15
:103760001BD0EDEC21F0070E03D0EDEC21F01F0E85
:10377000EE1603D0EDEC21F0EE52ED6A0DD0EDEC3B
:1037800021F0EE9E08D0EDEC21F00F0E03D0EDEC11
:1037900021F0070EEE16ED6AE9EC21F001E3DB2AD9
:1037A000FA2B88D7E552E7CFD9FF120001014E511D
:1037B00001E0CFD2E868521901E0B5D2E8685319A8
:1037C00001E0B1D2E868541901E0ADD2E8685519BA
:1037D00001E0A9D2100E4F1905E1FE0E501902E1C9
:1037E000010E511901E192D2140E4F1905E1F20EAA
:1037F000501902E1010E511901E175D2110E4F1954
:1038000005E1F20E501902E1010E511901E1F4D166
:10381000050E4F1905E1F20E501902E1010E511982
:1038200001E1D6D1010E4F1905E1F20E501902E166
:10383000010E511901E1B8D14F5105E1F20E5019B5
:1038400002E1010E511901E19BD10D0E4F1905E165
:10385000F10E501902E1010E511901E17DD1140E52
:103860004F1905E1F00E501902E1010E511901E165
:1038700036D14F5105E1EE0E501902E1010E5119FA
:1038800001E102D14F5101E047D2EE0E501901E0A3
:1038900043D2515101E040D2585101E1D3D05851A7
:1038A000080802E2BEEF20F058C1E6FF590EE66EAE
:1038B000010EC9EC21F00101590ED96FFB6B01011A
:1038C00058510101FB5D01E3BAD026EC22F0010A58
:1038D00001E1ADD0070A01E1AAD00C0A01E1A7D0AD
:1038E000030A01E18ED0010A01E17AD00F0A67E0F4
:1038F000020A55E0010A3FE0070A2CE0010A01E054
:103900009CD0000164514D6E4E6A030ED8904D3626
:103910004E36E804FBE1E00E00016315E00BE838E9
:10392000E84001014D10DA6F4EC0DBF1FAEC21F0F6
:10393000FF0EEE1802E1070EED1801E17ED0FAEC61
:1039400021F031EC22F0DA514D1802E1DB514E1832
:1039500074E069D0070E0001651540EC22F0070EF7
:10396000EE1801E1ED5069E03DEC22F002E150502B
:103970004E1863E058D000016551E840E840E84047
:103980001F0B40EC22F01F0EEE1801E1ED5055E048
:103990003DEC22F002E150504E184FE044D066C09A
:1039A000DAF1FAEC21F0FF0EEE1801E1ED5045E0FE
:1039B0003DEC22F002E150504E183FE034D00001BF
:1039C00067417F0B40EC22F07F0EEE1801E1ED50D5
:1039D00034E03DEC22F002E150504E182EE023D0AE
:1039E0000F0E0001681540EC22F00F0EEE1801E1F9
:1039F000ED5023E03DEC22F002E150504E181DE066
:103A000012D0700E00016815E8380F0B40EC22F060
:103A1000070EEE1801E1ED5010E03DEC22F002E15E
:103A200050504E180AE098EC21F0030E03D098ECA9
:103A300021F0010EEF6E580ED96FFB2B40D7590EB7
:103A4000D95D04E1259200017A891200580ED95DF2
:103A500001E094D3ADEC21F001E090D336EC22F0FC
:103A60009C6F9D6B9E91A5EC21F058C19FF10101C7
:103A700033EC21F06EE0D0EC21F06BE0D7EC21F0DC
:103A800068E00101992B65D0585104E148C1B8F1B3
:103A900000017A8D0101580501E070D3590501E05C
:103AA0006DD3ADEC21F004E0FF0E695D01E066D35B
:103AB00001015A51010A07E0010A0AE148C1B8F1BF
:103AC00000017A8F120048C1B8F100017A8D12000E
:103AD000ADEC21F001E03CD136EC22F025D058517C
:103AE0001BE0580501E04AD3020E595D21E15A510D
:103AF0000101DA6FDB6B5BC14EF04D6A4D50DA139A
:103B00004E50DB13B60EDA1902E16E0EDB1904E03B
:103B1000DA1D05E1DB1D03E100017B8512007FEC6E
:103B200021F0140E9B6FF00E0CEC22F0A0830CD051
:103B3000ADEC21F001E022D37FEC21F0140E9B6F5D
:103B4000F00E0CEC22F0A093A095A0970101070EB7
:103B5000996F00017A8B12005851010A06E0010AA0
:103B600001E0120000017C8706D0590501E0F0D089
:103B70005AA103D000017C89120000017C87120049
:103B80005851010A06E0010A01E0120000017D859A
:103B900006D0590501E0DCD05AA103D000017D8791
:103BA000120000017D8512005851010A06E0010A49
:103BB00001E0120000017D8906D0590501E0C8D05E
:103BC0005AA103D000017D8B120000017D891200F3
:103BD0005851010A06E0010A01E0120000017D8D42
:103BE00006D0590501E0B4D05AA103D000017D8F61
:103BF000120000017D8D12005851020A37E0030ABD
:103C00000BE0010A01E0120000017E857E897E8DB5
:103C10007E877E8B7E8F12005951020A11E0030AC3
:103C200001E012000F0E5A175AA105D000017E873D
:103C30007E8B7E8F120000017E857E897E8D120034
:103C40000F0E5A175A51040A0DE0050A07E0010A3F
:103C500001E0120000017E857E87120000017E894E
:103C60007E8B120000017E8D7E8F120059050DE1C2
:103C7000020E5B5D0AE10F0E5A150101F86F0F0E7F
:103C800001015C150101F96F0ED0020E595D60E172
:103C90005B055EE10F0E5A150101F96F0F0E010170
:103CA0005C150101F86FF951040A15E0050A0BE0F3
:103CB000010A01E01200F8A103D000017E87120082
:103CC00000017E851200F8A103D000017E8B120056
:103CD00000017E891200F8A103D000017E8F12003E
:103CE00000017E8D12005851010A06E0010A01E030
:103CF000120000017F8305D059052AE15AA103D0A3
:103D000000017F85120000017F831200585101E0FD
:103D100035D200018781120020DB01E02FD29CDB2D
:103D20009F6BC3EF21F0525153115411551101E112
:103D30001200585101E022D210DB01E01FD2DFDA7D
:103D400017DB7BDB9E899E9B9E9D9E9F9F6B1BDB53
:103D500012004E0501E012D2100E4F1905E1FE0EC1
:103D6000501902E1010E511901E1DBD1140E4F1976
:103D700005E1F20E501902E1010E511901E1B6D12F
:103D8000110E4F1905E1F20E501902E1010E511901
:103D900001E178D1050E4F1905E1F20E501902E14B
:103DA000010E511901E152D1010E4F1905E1F20E38
:103DB000501902E1010E511901E12AD14F5105E1DB
:103DC000F20E501902E1010E511901E1DCD00D0E85
:103DD0004F1905E1F10E501902E1010E511901E1EF
:103DE00097D04F5101E0C4D1EE0E501901E0C0D17F
:103DF000515101E0BDD1B1DA01E0120037DB9C6F17
:103E00009D6B1BDBF3DA08080FE052510F0B09081A
:103E100003E10101060E07D092DA09E3B0DA07E305
:103E200052510F0B0101416F01019E9902D0010116
:103E30009E899E9B9E9D9E9F53C19FF10101535160
:103E400001E190D15351080801E298D153C1E6FF36
:103E5000540EE66E010E9DDA0101FB6B0101535118
:103E60000101FB5D49E2F2DA080A36E00C0A1EE0C5
:103E7000070A12E0020A0CE0030A0AE0070A08E057
:103E8000030A06E0010A04E00E0A02E0030A31E137
:103E90004FDA010EEF6E2DD0F80E0001651701010B
:103EA000A9DAEECF4DF0070E4D1411D0070E000128
:103EB000651701019FDAD5DA1F0E4D16000E4E165A
:103EC000030ED8904D364E36E804FBE14D5000010C
:103ED0006513ABDA6B830DD0F00E0001681701019A
:103EE00089DAEECF4DF00F0E4D14000168139DDA04
:103EF0006B850101FB2BB2D7B6D901E136D150DA7F
:103F000001E133D154DA01E130D10101992B2DD1F6
:103F10005351010801E232D1F2D90D0E9B6FF10E1F
:103F200001DA05E0010A0AE101019E9914D0EDD9F8
:103F30000501020E1E6F0501020E09D000DA09E329
:103F40001EDA07E397DA05011E6F50DA05012D6FBF
:103F500005D001019E899E9B9E9D9E9F01012EDAA8
:103F60000101535101E1FED054054AE12BDA55A17C
:103F700005D055C134F500016B8947D055C125F5F1
:103F800000016B8742D05351010801E2F7D0B7D945
:103F90009B6BF20E9C6F010E9D6F10DA27DA090AF7
:103FA00005E0010A0AE101019E9914D0AED905018C
:103FB000020E006F0501020E09D0C1D909E3DFD955
:103FC00007E358DA0501006F11DA05010F6F05D01C
:103FD00001019E899E9B9E9D9E9F0101535101E17F
:103FE000C1D054050DE1EED955A105D055C116F546
:103FF00000016B8D0AD055C107F500016B8B05D010
:104000000101A081A093A095A0970101070EACD05B
:10401000535101E0B3D073D9010E14DA03E0010A61
:1040200008E189D072D90401020E4E6F0401020E1C
:104030000BD085D901E28ED0A2D901E28BD01ADA59
:1040400004014E6FD3D90401726F89D0535101E03E
:1040500095D055D9050EF6D903E0010A08E16BD0D9
:1040600054D90001020ECF6F0001020E09D067D9AA
:1040700071E385D96FE3FED90001CF6FB7D9000195
:10408000DE6F6DD0535101E079D039D9110EDAD9F4
:1040900003E0010A14E14FD038D90301060EA26FE4
:1040A0000301060EB16F0301060EC06F0301060E79
:1040B000CF6F0301060EDE6F0301060E15D03FD948
:1040C00049E35DD947E3D6D90301A26F8FD9030134
:1040D000B16F8CD90301C06F89D90301CF6F86D925
:1040E0000301DE6F83D90301ED6F39D0535146E1EF
:1040F00006D9140EA7D903E0010A08E11CD005D99E
:104100000401060ED66F0401060E09D018D922E369
:1041100036D920E3AFD90401D66F68D90401E56F21
:104120001ED053512BE1EBD8100E9B6FFE0EFAD828
:1041300005E0010A07E101019E990ED0E6D80501CC
:10414000020E06D0FCD806E31AD904E393D9050180
:10415000536F05D001019E899E9B9E9D9E9F0101EC
:104160006CD99F6B0101060E996F00017A8B1200CA
:10417000F4D804E171D953C19FF105D91200D9CF08
:10418000E6FFE1CFD9FF010175515FE1765109E109
:10419000EE0E771906E1785104E1259200017A8943
:1041A00054D0765152E1EE0E77194FE1010E781995
:1041B0004CE180054AE101012F6BEE0E306F010EDC
:1041C000316F81C1CAF1FE0EDB50FF0823E1200EE2
:1041D0002A6F0101C269010EC66F0101CA050CE117
:1041E000130E01012B6F2C6B030E2D6F0101030EBB
:1041F000C76F00017B8128D0CA5127E12B0E010136
:104200002B6F2C6B070E2D6F0101070EC76F00017E
:104210007B831AD0FE0EDB500001695D16E10101BF
:10422000100E2A6F0101CA0506E1130E01012B6F62
:104230002C6B030E07D0CA5106E12B0E01012B6F28
:104240002C6B070E2D6F00017A85E552E7CFD9FF61
:104250001200E96EEA6AD890E936EA36E30EE926FA
:10426000010EEA221200F15101010F0BF36EF00E64
:10427000A015F310A06F0101F2510101BED8A015E5
:10428000F310A06F0101F35101010F0BF36EF00E5B
:10429000A115F310A16F0101F4510101AED8A115D0
:1042A000F310A16F0101F55101010F0BF36EF00E38
:1042B000A215F310A26F0101F65101019ED8A215BB
:1042C000F310A26F0101F75101010F0BF36EF00E15
:1042D000A315F310A36F0101F85101018ED8A315A6
:1042E000F310A36F0101070E996F0101A1510F0B8C
:1042F0000F0812008AD8EF50E66EFA51120048C13A
:1043000093F10101020E9A6F120001019E999E9B8A
:104310009E9D9E9F1200A5D8DA514F6E506A4F5055
:104320004D1812009C6F010E9D6F60D8090A120093
:10433000FB51EA6AF10FE96E010EEA2212005251B6
:104340000F0B4D6E000E4D5C12009E939E959E9736
:104350009E999E9B9E9D9E9F1200000169510101A6
:10436000695D1200EA6ADC0FE96E010EEA221200B2
:104370004FC19BF150C19CF151C19DF112005251AE
:104380000F0B070812000101060E996F00017A8BCE
:104390001200E66E54EC1BF0E552E552E5521200B5
:1043A0000101992B0101A2510F0B0F08120001010D
:1043B000992B0101A3510F0B0F0812003ED853C1D6
:1043C0009FF112000101A091A093A095A097010177
:1043D0001200FD0EDB2AFE0E12008CDF3ADFE552E2
:1043E000E750EE6EED6AFA5129EF21F001015251CA
:1043F0000F0B1200FB5129EF21F00F0BF36EF34668
:10440000F346F346F3460F0E1200FD0EDBCFE9FF35
:10441000FE0EDBCFEAFF12009C6F010E9D6F9E9196
:1044200094DF010E9F6FA0811200010181DFEF6A0E
:10443000259200017A89000112009E919E939E951B
:104440009E9712009B6FF20E92EF21F071DFEF6AE0
:10445000FB5188DFEF50120052DF8ADF9E81A5EF0B
:1044600021F0EECF4DF0EFCF4EF0120048DF9B6B06
:10447000EE0E12004ADFF6EF21F0BCDF8BEF21F0E9
:084480000101DA6FFAEF21F0EF
:08448800ECEC27F00001606B71
:104490007A6B7B6B7C6B7D6B7E6B7F6B806B816BD8
:1044A000826B836B846B856B866B876B886B2594C3
:1044B00025962598259C259E6B6BFD0EDBCF69F01C
:1044C000FD0EDBCF6AF0F80EDB500F0B4D6EF90ED0
:1044D000DB500F0B100DF3504D10616FFA0EDB50D7
:1044E0000F0B4D6EFB0EDB500F0B100DF3504D10EC
:1044F000626FFC0EDB501F0B4D6EA00E4D10636FF4
:10450000400E646FF70EDBCF65F0A00E666F640E91
:10451000676FF60EDB500F0BC009686FFE0EDB50A5
:1045200002E1E66A02D0600EE66E29EC31F0E55257
:1045300003EC34F075EC28F000017A89258025928F
:10454000020EC66F110EBF6F020EC76F110EC06F45
:104550000A0EC86F110EC16F020EC96F110EC26F25
:10456000320ECA6F110EC36F1E0ECB6F110EC46FC9
:10457000040ECC6F110EC56FB36BB46BB56BB66B1D
:10458000B76BB86BB96BBA6BBB6BBC6BBD6BBE6BFF
:10459000A783A795A787A799A78BA79DA885A89765
:1045A000A889A89BA88DA89F29EC28F0AA83AA9582
:1045B000AB89AB9BAD81AD93AD87AD99B085B0971D
:1045C000B099B08DB09FB181B193B195F1EF27F063
:1045D000ECEC27F00001070EA66FA63525E2A6C079
:1045E000E9FFEA6AE9BEEA68F5EC27F04EBE4F68DB
:1045F000FFEC27F04D5C02E2010E16D0A6C0E9FFE9
:10460000EA6AE9BEEA68F5EC27F04EBE4F68FFECB7
:1046100027F0D8804D5404E3A65104E1070E606FE3
:10462000000E02D0A607D9D7F1EF27F0ECEC27F067
:1046300030EC28F0CDDFE552E552000906E0258098
:10464000259200017A89560E20D0000169514D6EE5
:104650004E6AD8904E5004E6FB0E4D5C000E4E584C
:1046600002E2692B01D0696B6A51695D05E0258022
:1046700025927A89550E09D0FE0E696F2584258012
:1046800025927A89060E606F570EF1EF27F0D9CF89
:10469000E6FFE1CFD9FFFD0EDBCFE9FFFE0EDBCF5A
:1046A000EAFF050EE926000EEA22EF501F0B57E144
:1046B000FD0EDBCFE9FFFE0EDBCFEAFF030EE9269E
:1046C000000EEA22EF50E66EFB0EDBCFE9FFFC0E98
:1046D000DBCFEAFFE552E750EF6EFD0EDBCFE9FFDF
:1046E000FE0EDBCFEAFF050EE926000EEA22EF50B0
:1046F000E66EFB0EDBCFE9FFFC0EDBCFEAFF030E1D
:10470000E926000EEA22E552E750EF6EFB0EDBCF02
:10471000E9FFFC0EDBCFEAFF050EE926000EEA22D8
:10472000EF6AFD0EDBCFE9FFFE0EDBCFEAFF050EE1
:10473000E926000EEA22010EE926000EEA22EF50D9
:10474000E66EFB0EDBCFE9FFFC0EDBCFEAFF040ECB
:10475000E926000EEA22E552E750EF6E44D0FB0E48
:10476000DBCFE9FFFC0EDBCFEAFFEFCF4DF0FD0E14
:10477000DBCFE9FFFE0EDBCFEAFF030EE926000EDA
:10478000EA22EF504D5C2AE1FB0EDBCFE9FFFC0E85
:10479000DBCFEAFF030EE926000EEA22EF2AFB0E2A
:1047A000DBCFE9FFFC0EDBCFEAFF030EE926000EAC
:1047B000EA22EFCF4DF0FD0EDBCFE9FFFE0EDBCF9F
:1047C000EAFF050EE926000EEA22EF504D5C05E0F7
:1047D0000001040E606F010E92D005D00001050E9D
:1047E000606F010E8CD00001010EA56F080E000154
:1047F000A55D01E382D00001A5050FE1FB0EDBCF33
:10480000E9FFFC0EDBCFEAFF030EE926000EEA22E9
:10481000EF501F0B02E100006DD0FD0EDBCFE9FF72
:10482000FE0EDBCFEAFF050EE926000EEA22E9CFF5
:104830004FF0EACF50F00001A5510F014F24E96E6F
:10484000000E5020EA6EEF50E66EFB0EDBCFE9FF64
:10485000FC0EDBCFEAFF050EE926000EEA22EF5040
:104860004D6E4E6AFB0EDBCFE9FFFC0EDBCFEAFF9D
:10487000EE524D50EE24E76E4E50EE20EA6EE7CF3A
:10488000E9FFE552E750EF6EFB0EDBCFE9FFFC0ED0
:10489000DBCFEAFF050EE926000EEA22EF2AFB0E27
:1048A000DBCFE9FFFC0EDBCFEAFF050EE926000EA9
:1048B000EA22EFCF4DF0FB0EDBCFE9FFFC0EDBCFA2
:1048C000EAFF040EE926000EEA22EF504D5C10E2EA
:1048D000FB0EDBCFE9FFFC0EDBCFEAFF050EE9267E
:1048E000000EEA22EFCF4EF0FA0EDB504E5C02E3F0
:1048F0005A0E05D00001A52B79D75B0E00D0E552EA
:10490000E7CFD9FF120068DBB2DBEF50080B01E004
:104910000BD17FDBEE0A01E1F5D0020A74E0070A51
:1049200019E0010A01E017D130DBEFCF0FF147DBCF
:10493000EFCF1AF126DBEFCF12F123DB010E9EDB66
:10494000EFCF13F11EDB020E99DBEFCF14F1ACECCD
:104950001AF003D10001946B080E945D01E3FDD0C1
:1049600094510DE1902B0DDB64DB905D02E00B0EAA
:10497000C7D00BDBEF50915D44E00A0EC1D08951E6
:104980008B5D8A518C593DE28D5139E1ED0E8E19C6
:1049900036E1010E8F1933E192DB4BDBE66E750ECB
:1049A0008B25E96E010E8C21EA6EE552E750EF6E21
:1049B0008B2B000E8C2389518B1923E18A518C1982
:1049C00020E16951925D15E1E0DAEFCF35F10101A7
:1049D0003D69130E396F8DC03EF18EC03FF18FC01F
:1049E00040F11CC13AF11DC13BF190C03CF1000106
:1049F0007A8792C0E6FFBFEC20F0E552AED0090EF8
:104A00007FD0942BA9D7BDDAEFCF1BF1BADA010E14
:104A100035DBEFCF1CF1B5DA020E30DBEFCF1DF145
:104A2000B0DA030E2BDBEFCF1EF1ABDA040E26DB80
:104A3000EFCF1FF1A6DA050E21DBEFCF20F1A1DACF
:104A4000060E1CDBEFCF21F19CDA070E17DBEFCF50
:104A500022F10001906B8B6B8C6B20C18DF021C11A
:104A60008EF022C18FF091DAEFCF91F0A8DAEFCF7C
:104A700092F001011B51130A70E0020A26E0010ABC
:104A80000BE0300A6AE10101266901012E691CC1AF
:104A900089F01DC18AF061D01CC189F01DC18AF066
:104AA0000101110E2A6F2D692E69010E2C6F1EC196
:104AB0002BF120C12FF121C130F122C131F165DA92
:104AC000EFCF26F100017A8548D0205117E1EE0E94
:104AD000211914E1010E221911E11DC1C6F11CC1F9
:104AE000C7F191C0C2F10101CA0503E100017B8158
:104AF00034D0CA5132E100017B832FD000010C0E6B
:104B0000606F2BD042DAEF500001695D26E13DDA9B
:104B1000EF50FE0822E0D3DAE9CFE6FFEACFE6FF66
:104B200085DDE552E5521AD074DAED0814E147DA72
:104B3000EFCF69F11B0EE66E480EE66E010EE66ED3
:104B40008FDAA5DD4D6E050EE15E4D505A0805E188
:104B5000D6EC1BF002D05C0E01D0000E42D23CDA43
:104B60002550010B01E056D12550020B01E052D136
:104B70002550040B01E04ED10001B351B411B51121
:104B8000B61101E12ED1B35125DA00092FE0CD6B2A
:104B900044DA06E2BF51000801E2BF07CD2BF8D787
:104BA000BF5124E1C6C0BFF090DAEF5013DA49DA02
:104BB00002E04BDAFEE1E8508FDA0001A7510ADA91
:104BC000000902E1A787A799B35104DA4D6EA751F6
:104BD00001DA4D14E9E0A751FDD94D6E7C0EE96E66
:104BE000000EEA6EEF50F6D94D1076DAB45119DAAC
:104BF00000092FE0CD6B11DA06E2C051000801E296
:104C0000C007CD2BF8D7C05124E1C7C0C0F0D1D91F
:104C1000EF5007DA16DA02E018DAFEE1E850C3D9FD
:104C2000F30EBCD90001A851FCD9000902E1A88506
:104C3000A897B451F6D94D6EA851F3D94D14E7E0B9
:104C4000A851EFD9C0D9EF50ECD94D10ACD9F30E23
:104C5000A5D9B451B1D900092BE0CD6BDED906E25C
:104C6000C151000801E2C107CD2BF8D7C15120E1A5
:104C7000C8C0C1F09ED9EF509FD9E3D902E0E5D971
:104C8000FEE1E8500FDA0001A85196D9000902E1CF
:104C9000A889A89BB45190D94D6EA8518DD94D14B7
:104CA000E9E0A85189D98FD9EF5086D94D10FAD9AA
:104CB000B4516FD900092BE0CD6BAFD906E2C251D8
:104CC000000801E2C207CD2BF8D7C25120E1C9C0CC
:104CD000C2F06FD9EF505DD9B4D902E0B6D9FEE188
:104CE000E850D0D90001A85154D9000902E1A88D9B
:104CF000A89FB4514ED94D6EA8514BD94D14E9E03F
:104D0000A85147D960D9EF5044D94D10BBD9B551FE
:104D10008CD900092CE0CD6B80D906E2C351000884
:104D200001E2C307CD2BF8D7C35121E1CAC0C3F0BC
:104D300040D9EE52EF5079D984D902E086D9FEE10C
:104D4000E850A8D90001A95170D9000901E181D921
:104D5000B5516BD94D6EA95168D94D14E9E0A951EF
:104D600064D931D9EE52EF5060D94D1093D9B65174
:104D7000060BE842000935E0CD6B4FD906E2C4517D
:104D8000000801E2C407CD2BF8D7C4512AE1CBC0FB
:104D9000C4F00FD9EE52EE52EF50060BE84251D953
:104DA00002E053D9FEE1E85083D90001AA51060B75
:104DB000E842000902E1AA83AA95B651060BE8422F
:104DC0004D6EAA51060BE8424D14E3E0AA51060BC2
:104DD000E842F9D8EE52EE52EF50060BE8424D1081
:104DE00067D9B751B811B911BA11BB51BC11BD1176
:104DF000BE1110E0BEA10ED0CD6B0FD906E2C55199
:104E0000000801E2C507CD2BF8D7C55103E1CCC09E
:104E1000C5F08781E6D077A224D07792779000EC16
:104E200032F000016C6FE850010A03E0030A01E070
:104E30001200C00EF214CE6F3F0EF2166D0EE66E2B
:104E4000000EE66E07EC33F0E552E5526D0EE66EAD
:104E5000000EE66E58DDE552E5520001CE51F21229
:104E6000120077A803D0779895EC32F0120025BC99
:104E700080D025B219D000017A517B1112E10001D6
:104E80007C517D117E117F110CE100018051811157
:104E90008211831106E10001845185118611871169
:104EA00002E079EC29F039D025A637D0259600010B
:104EB000030E936F0001935100082FE20001882B2D
:104EC000000188514D6E4E6AD8904E5004E6FA0E9D
:104ED0004D5C000E4E581EE30001886BC00EF214AC
:104EE0000001CE6F3F0EF216259225B40BD025900F
:104EF00069C0E6FF80EC33F0E55269C06AF000015A
:104F00006B8104D0E66880EC33F0E5520001CE51AD
:104F1000F21203D000019307CDD7035000081AE224
:104F2000C00EF2140001CE6F3F0EF216980EE66E20
:104F3000000EE66E07EC33F0E552E552980EE66E91
:104F4000000EE66EE0DCE552E5525C0800E100018F
:104F5000CE51F21202019EA105D002019E910001E4
:104F6000030E606F71AA04D0258C0001020E606FE1
:104F700007D025BE03D0258E6F8802D06FA8FF0012
:104F8000120075D8050E3EEF28F071D8030E3EEFE3
:104F900028F0C00BE842E842E842A3D0EF14F31037
:104FA000EF6EF4501200030BF36EF46EF346F3460B
:104FB00012008BD8EE521200300BE84292D057D834
:104FC000020E3EEF28F04D6E7C0EE96E000EEA6E8A
:104FD000EE521200180B85D0D9CFE6FFE1CFD9FFF2
:104FE0001200E552E7CFD9FF1200610EE926000E4C
:104FF000EA22EFCF4DF0A6C04EF04F6A1200FD0E30
:10500000DB504E24E96EFE0EDB504F20EA6EEF506F
:1050100012002DD8EE52EF501200FE0EDB50CD5D87
:1050200012000C0BE842E8421200FC0BE842E84296
:1050300012009451E924E96E000EEA20EA6EEF5066
:1050400012004DC0E7FFE7521200E846FE0BE706EC
:105050001200A985A997A999A99BA99DA99F1200AA
:10506000FD0EDBCFE6FFFE0EDBCFE6FF1200FD0EEE
:10507000DBCFE9FFFE0EDBCFEAFF1200E926000ED0
:10508000EA22120090DFF346F346F346F3463F0E62
:10509000CEEF27F03F0BF36EF46EF346F346030EAC
:1050A000CEEF27F080DFF346F346CF0ECEEF27F0AA
:1050B000030BF36EF46EF346F90ECEEF27F061DFCB
:1050C000E9CF4DF0EACF4EF01200010E4D6EA70E63
:1050D000E96E000EEA6E120066DFF346E70ECEEFD1
:0A50E00027F0E842E842E84212001F
:0650EA001200D9CFE6FF21
:1050F000E1CFD9FFC0EC2DF0E8B03C87C8EC2DF033
:10510000B1EC2DF0EFCF41F5B1EC2DF0010EB8EC84
:105110002DF0EFCF42F5B1EC2DF0AEEC2DF0EFCF4E
:1051200043F5B1EC2DF0030EB8EC2DF0EFCF44F5C4
:10513000B1EC2DF0040EB8EC2DF0EFCF45F5B1EC4D
:105140002DF0050EB8EC2DF0EFCF46F5B1EC2DF0BB
:10515000060EB8EC2DF0EFCF47F5B1EC2DF0070EB1
:10516000B8EC2DF0EFCF48F566EC2DF0E552E7CF27
:10517000D9FF1200D9CFE6FFE1CFD9FF040EE12617
:10518000B5EC2DF001E190D0B5EC2DF0060802E36E
:10519000010E1FD0B5EC2DF00D0802E3020E19D060
:1051A000B5EC2DF0140802E3030E13D0B5EC2DF08E
:1051B0001B0802E3040E0DD0B5EC2DF0220802E32B
:1051C000050E07D0B5EC2DF0290802E3060E01D03C
:1051D000070EF36E030EF3CFDBFFDF6A020EDB6A0E
:1051E000030EDB50F36E020EDBCFF4FFF350F45CE2
:1051F0004FE2C0EC2DF0E8B03C87C8EC2DF04091B8
:10520000409340954087010EDB6A080EF36E010E55
:10521000DBCFF4FFF350F45C36E2010EDB5009E122
:10522000BCEC2DF0EF5060EC2DF0BCEC2DF0EF2A33
:1052300027D0010EDB0408E1020EDB5005E1B5ECDE
:105240002DF060EC2DF01CD0B5EC2DF0DF5C15E2FC
:10525000DF504D6E4E6A3CEC2DF0050EB8EC2DF093
:105260004D50EE24E76E4E50EE20EA6EE7CFE9FF98
:10527000EF5060EC2DF0DF2A03D0CFEC2DF0EF687B
:10528000010EDB2AC2D766EC2DF0020EDB2AA8D76E
:10529000200E4D6EBCEC2DF04D50EF26E00E4D6E05
:1052A000BCEC2DF04D50EF16040EE15C02E2E16A19
:1052B000E552E16EE552E7CFD9FF12000501506BD0
:1052C000516B000E505D0D0E515909E266EC2DF048
:1052D000000905E00501502B000E5123F2D705010E
:1052E000505106E10D0E511903E10001080E606FE7
:1052F0001200065001E0120000017A517B1160E0BB
:105300007AAB0AD025B85BD0900EE66E010E90EC19
:105310002DF000017A9B49D07AA707D0320EE66EB5
:10532000010EC4DB00017A9712007AA507D0230E84
:10533000E66E010EBBDB00017A9512007AA90DD052
:10534000410EE66E010EB2DB25B404D00001886B7D
:105350002580258200017A9912007AA107D0000EDB
:10536000E66E010EA3DB00017A9112007BA506D048
:1053700025B825D0E1D800017B9517D07AAD06D0AD
:1053800025B81DD0B1D900017A9D0FD07AAF06D0D3
:1053900025B815D063DA00017A9F07D07BA107D02A
:1053A00025B80DD0FED900017B91258812007BA382
:1053B000C2D025B8C0D0D7DA00017B93258812006F
:1053C000065001E0B8D02550010B01E0B4D02550C3
:1053D000020B01E0B0D02550040B01E012000001E7
:1053E0007C517D117E117F1101E18FD07CA707D008
:1053F0001E0EE66E050E5ADB00017C9712007CA99A
:1054000007D02D0EE66E050E51DB00017C991200CF
:105410007DA507D0000EE66E050E48DB00017D95E8
:1054200012007DA707D00F0EE66E050E3FDB0001D0
:105430007D9712007DA909D025B87DD04E0EE66E6D
:10544000040E6EDB00017D990AD07DAB0AD025B831
:1054500072D0720EE66E040E63DB00017D9B258820
:1054600012007DAD07D0CF0EE66E000E1FDB0001EF
:105470007D9D12007DAF07D0DE0EE66E000E16DBBE
:1054800000017D9F12007EA506D0A20EE66E030EDF
:105490008EDB7E9512007EA706D0B10EE66E030E5F
:1054A00086DB7E9712007EA906D0C00EE66E030E44
:1054B0007EDB7E9912007EAB06D0CF0EE66E030E29
:1054C00076DB7E9B12007EAD06D0DE0EE66E030E0E
:1054D0006EDB7E9D12007EAF06D0ED0EE66E030EF3
:1054E00066DB7E9F12007FA307D0D60EE66E040E09
:1054F000DDDA00017F9312007FA51DD0E50EE66E78
:10550000040ED4DA00017F95120000018051811150
:105510008211831101E0120000018451851186116E
:10552000871109E087A107D0530EE66E050EBEDA9B
:10553000000187911200120005014D6B140E4D5DA4
:1055400001E3CCD00101CB519EDA3C87F00E3D6FD8
:10555000140E3E6F69C03FF50101D751D72B0501ED
:10556000416F4D51130A01E1B1D0010A01E1A6D00A
:10557000030A01E1A3D0010A01E1A0D01F0A01E161
:105580009DD0010A01E17CD0030A01E197D0010A14
:1055900001E194D0070A01E191D0010A6AE0030A0F
:1055A00060E0010A01E18AD00F0A01E187D0010A17
:1055B00001E184D0030A49E0010A41E0070A31E031
:1055C000010A21E0030A11E0010A01E083D0860EFE
:1055D000426F150E436F050E446FB60E456F6E0E8B
:1055E000466F520E476F530E67D0310E426F310E29
:1055F000436F200E446F450E456F6E0E466F670E6B
:10560000476F690E59D06E0E426F650E436F200EC4
:10561000446F440E456F610E466F740E476F610E06
:105620004BD0200E426F430E436F6F0E446F6E0ED1
:10563000456F760E466F650E476F720E3DD0740E45
:10564000426F650E436F720E19D0426B436B330E7F
:10565000446F2E0E456F350E466F300E476F200E8D
:105660002BD0426B436B446B456B466B476B340EE0
:1056700023D0610E426F310E436F310E446F21D043
:10568000426B436B446B000162390F0B0F0B300F01
:105690000501456F0F0E00016215300F0501466FC1
:1056A000000161390F0B0F0B300F0501476F0F0E13
:1056B00000016115300F0501486F0CD0426B436B40
:1056C000446B456B466B476B486B04D0426B010ED5
:1056D000436F2CDAF3DD05014D2B30D7200E01018D
:1056E000D727E00ED71712000501496B030E495D5D
:1056F00057E260DA4951150A48E0010A46E0070A14
:1057000044E0010A42E0030A40E0010A3EE01F0AC9
:105710003CE0010A3AE0030A38E0010A36E0070AF1
:1057200034E0010A32E0030A30E0010A2EE00F0AF9
:105730002CE0010A2AE0030A28E0010A26E0070A11
:1057400024E0010A18E0030A0CE0010A25E1130E27
:10575000FBD9446BE80E456F466B476BEA0E486F0A
:105760001BD0426B436BEB0E446F456B466BEC0EEC
:10577000476F486B11D0426BEE0E436F446B456B25
:10578000ED0E466F010E476F06D0426943694469CA
:10579000456946694769486991DD0501492BA6D7E6
:1057A000D7D1CAD9C6C14BF54F514B5D56E207DA86
:1057B0004B51160A47E0030A45E0010A43E0070A95
:1057C00041E0010A3FE0030A3DE0010A3BE01F0A15
:1057D00039E0010A37E0030A35E0010A33E0070A3D
:1057E00031E0010A2FE0030A2DE0010A2BE00F0A45
:1057F00029E0010A27E0030A25E0010A23E0070A5D
:1058000018E0010A0CE0030A24E1010E426F436B29
:10581000E80E446F456B466BEA0E476F08D0426B4B
:10582000EB0E436F446B456BEC0E466F476B486B5A
:1058300010D0EE0E426F436B446BED0E456F010EC0
:10584000466F05D0426943694469456946694769BD
:10585000486934DD05014B2BA7D7120005014A6BBF
:10586000070E4A5D01E37ED0A5D94A51150A73E0BF
:10587000010A71E0070A6FE0010A6DE0030A6BE0BC
:10588000010A69E01F0A67E0010A65E0030A63E0B4
:10589000010A61E0070A5FE0010A5DE0030A5BE0DC
:1058A000010A59E00F0A57E0010A52E0030A41E0F9
:1058B000010A33E0070A26E0010A18E0030A0CE0B7
:1058C000010A4CE12B0E426F436B446BE80E456FAF
:1058D000466B476BEB0E3AD0426B436BEC0E446F5A
:1058E000456B466BEE0E476F486B38D0426BED0E42
:1058F000436F010E446F456BEE0E466F010E476F0E
:10590000140E24D0F00E20D90D0E446FF10E456F09
:10591000010E466F476BF20E19D0010E15D9F20E2B
:10592000446F010E456F050E466FF20E476F010E74
:105930000DD0110E426FF20E436F010E446F140E24
:10594000456FF20E466F010E476F100E486F06D07E
:10595000FE0EFAD802D042694369E8D8AFDC0501EF
:105960004A2B7ED7F5D0E8D8C6C14CF54F514C5DD7
:1059700001E381D024D94C51160A75E0030A71E085
:10598000010A6FE0070A6DE0010A6BE0030A69E0B3
:10599000010A67E01F0A65E0010A63E0030A61E0AB
:1059A000010A5FE0070A5DE0010A5BE0030A59E0D3
:1059B000010A57E00F0A52E0010A43E0030A33E00C
:1059C000010A24E0070A17E0010A0BE0030A4EE18E
:1059D000426B436BE80E446F456B466BEB0E476FB3
:1059E00008D0426BEC0E436F446B456BEE0E466F76
:1059F000476B486B3BD0ED0EA7D8446BEE0E456F5E
:105A0000010E466F140E476FF00E26D0010E426F46
:105A10000D0E436FF10E446F010E456F466BF20E93
:105A2000476F010E19D0010E426FF20E436F010E47
:105A3000446F050E456FF20E466F010E476F110E53
:105A40000BD0F20E81D8140E446FF20E456F010E8A
:105A5000466F100E476FFE0E486F08D0010E426F62
:105A600003D0426901D04269436960D85EEC29F0F5
:105A700005014C2B7BD71200FD0EDBCFE9FFFE0E9C
:105A8000DBCFEAFF12000501070BF36EF346F34686
:105A9000F346F346F3461F0E3C15F3103C6F12001D
:105AA00067D8EE50EFCFEAFFE96E1200E66E76ECB3
:105AB00028F0E552E5521200090E5AD8EF501200B4
:105AC000E66E6DD8E552E750EF6E12003C0EE66EC2
:105AD000050EE66EDEEC32F0E552E55212003C8730
:105AE000EE0E3D6FB8C13EF569C03FF50101D651DC
:105AF000D62B0501416F12003C97EB0E3D6FC2C1E2
:105B00003EF569C03FF50101C651C62B0501416F45
:105B10001200030E2DD8EFCF3EF569C03FF51200FD
:105B2000E66EBAEC28F0E552E55212004469456988
:105B30004669476948691200C6C14EF50101C65160
:105B4000C72505014F6F1200426F010E436F12000F
:105B5000200E0101D627E00ED6171200020EB8EF74
:105B60002DF08ADF050E50EF2DF086DF5CEF2DF073
:105B7000E926000EEA2212007FDF070E50EF2DF01B
:105B80007BDFEF5080DF78DFEE52EF503C97120062
:105B900073DFE4DFEFCF3DF56FDF89EF2DF0010E0E
:105BA000DB50EA6A410FE96E050EEA2212007EDF41
:105BB000000112000101B55166DF6FEF2DF0010108
:085BC000BF5161DF7CEF2DF005
:085BC800325001E18CD0325093
:105BD000010B03E13250020B25E032A007D0050192
:105BE0006451EA6A000FE96E030E06D005016451A4
:105BF000EA6A170FE96E030EEA22EFCF6EF5642B07
:105C00006451160807E36E5102E06EC5ADFF0A0E3F
:105C10006E5D68E132A003D062913290120062930F
:105C20003292120032A417D005016551EA6A2E0F94
:105C3000E96E030EEA22EFCF6EF5652B65513E0843
:105C400007E36E5102E06EC5ADFF0A0E6E5D4AE1DC
:105C50006295329412003250080B03E13250100B5F
:105C600025E032A607D005016651EA6A6D0FE96E9C
:105C7000030E06D005016651EA6A7F0FE96E030E36
:105C8000EA22EFCF6EF5662B6651110807E36E51DD
:105C900002E06EC5ADFF0A0E6E5D24E132A603D0B0
:105CA00062973296120062993298120032AA17D087
:105CB00005016751EA6A910FE96E030EEA22EFCF00
:105CC0006EF5672B6751100807E36E5102E06EC551
:105CD000ADFF0A0E6E5D06E1629B329A120032AE93
:105CE00020D012001200050162A103D0646B328043
:105CF000120062A303D0646B3282120062A503D04B
:105D0000656B3284120062A703D0666B3286120084
:105D100062A903D0666B3288120062AB02D0676B57
:105D2000328A120031A207D031A603D031963192C7
:105D300022D0318622D00501635103E10001605178
:105D400018E0318263C5E6FF6BDA26C099F327C0FD
:105D50009AF30501636B60C0E6FF62DA26C09DF32B
:105D600027C09EF30001606B0501628B8B8A8B88D4
:105D700004D031B202D08B9A8B98080402E18BAA2E
:105D80008B8812000501300E6A6F300E6B6F300E7B
:105D90006C6F300E6D6F800E69153AE1D8906951C5
:105DA00004E6100E685D270E695906E3100E685F61
:105DB000270E695B6A2BF2D7D890695104E6E80E8A
:105DC000685D030E695906E3E80E685F030E695BC0
:105DD0006B2BF2D7640E69AF02D0D89003D0685D08
:105DE000000E695906E3640E685F000E695B6C2B58
:105DF000F1D70A0E69AF02D0D89003D0685D000ECB
:105E0000695906E30A0E685F000E695B6D2BF1D7D6
:105E1000120032BE33D10850050A01E1A0D00F0AAA
:105E200001E19DD0080A51E0050A4FE0060A03E0AF
:105E3000070A01E0120007A027D007C52DF0F4D90A
:105E400005E12A6A300E2B5C01E12B6A2AC009F3B6
:105E50002BC00AF32CC00BF308C56FF509C570F50C
:105E6000020E0F0B050105E0D89070336F33E80682
:105E7000FBE1DFD929C00DF32AC00EF32BC00FF3CD
:105E80002CC010F30501628107A4F8D007C52DF0DE
:105E9000CBD905E12A6A300E2B5C01E12B6A2AC0BE
:105EA00074F32BC075F32CC076F361C468F562C43B
:105EB00069F568DF6AC578F36BC579F36CC57AF369
:105EC0006DC57BF305016287120007A227D016C5B6
:105ED0002DF0AAD905E12A6A300E2B5C01E12B6A6C
:105EE0002AC020F32BC021F32CC022F317C56FF575
:105EF00018C570F5020E0F0B050105E0D890703340
:105F00006F33E806FBE195D929C024F32AC025F3B5
:105F10002BC026F32CC027F30501628307A6AED061
:105F200016C52DF081D905E12A6A300E2B5C01E1FE
:105F30002B6A2AC086F32BC087F32CC088F385C454
:105F400068F586C469F51EDF6AC58AF36BC58BF3F5
:105F50006CC58CF36DC58DF30501628912002CC4EC
:105F60002DF02BC42EF085EC36F029C035F32AC075
:105F700036F32BC038F32CC039F32EC42DF02DC4CA
:105F80002EF085EC36F029C03BF32AC03CF32BC041
:105F90003EF32CC03FF330C42DF02FC42EF085EC1F
:105FA00036F029C041F32AC042F32BC044F32CC081
:105FB00045F332C42DF031C42EF085EC36F029C003
:105FC00047F32AC048F32BC04AF32CC04BF334C428
:105FD0002DF033C42EF085EC36F029C04DF32AC0E5
:105FE0004EF32BC050F32CC051F336C42DF035C402
:105FF0002EF085EC36F029C053F32AC054F32BC0A1
:1060000056F32CC057F366C4E6FF0AD926C059F3ED
:1060100027C05AF365C4E6FF03D926C05BF327C047
:106020005CF364C4E6FFFCD826C05DF327C05EF3D2
:1060300063C4E6FFF5D826C05FF327C060F38AC4C7
:10604000E6FFEED826C062F327C063F389C4E6FFFB
:10605000E7D826C064F327C065F388C4E6FFE0D81C
:1060600026C066F327C067F387C4E6FFD9D826C0E9
:1060700068F327C069F30501628512001200A8D8F1
:10608000E652DEEC05F0E552B8D81100D8CFE4FFB7
:10609000E0CFE4FFE46E9CD800EE39F0140EE80483
:1060A00003E3EECFE4FFFBD700EE4DF00D0EE80466
:1060B00003E3EECFE4FFFBD7E65259EC06F00BEC1E
:1060C00027F09EAA16D0AE50366EAB50040B03E1FB
:1060D000AB50020B05E0AB98AB880501020E636F75
:1060E000400E365C02E1318804D031A802D038EC91
:1060F00018F0E55200EE59F00D0EE80403E3E5CF89
:10610000EDFFFBD700EE4CF0140EE80403E3E5CFFF
:10611000EDFFFBD772D8E550E5CFE0FFE5CFD8FF24
:106120001000806A816A0A0EE66EE66AB7EC3AF001
:10613000E552E552F009E81C826EBF0E926EBF0E6A
:10614000936E400E946E8B888B8ACC0EE66E93EC29
:106150003BF0E552400EE66E030EE66E4C0EE66E28
:1061600046EC3AF0E552E552E552316A0501626BC0
:10617000326A636BD0B602D0010E636FF26A800E92
:10618000F16EF06A9F9A9D8AD08ED6EC12F0B5EC33
:106190000CF01CEF00F0C5DF0400D1809E6AA16AFC
:1061A000A46AB76A776AC00EF212CD80CA84B18041
:1061B00037EC27F02EEC04F0085006E00400B2DDC6
:1061C00006EC11F026DE086AACB2FEDCF1D7120054
:1061D000DACFE4FFE2CFDAFFE9CFE4FFEACFE4FF72
:1061E000F6CFE4FFF7CFE4FFF5CFE4FFF3CFE4FF12
:1061F000F4CFE4FFFACFE4FF1200E5CFFAFFE5CFDA
:10620000F4FFE5CFF3FFE5CFF5FFE5CFF7FFE5CFEF
:10621000F6FFE5CFEAFFE5CFE9FFE5CFDAFF1200B1
:106220000BEC36F0E55212005EEC36F0300E2A5CD4
:0E62300012006FC52DF070C52EF085EF36F010
:02623E00016AF3
:106240000268036A120002019C6B046A0568066A10
:106250001200ADDAFE0EDBCF9DF202019E6B9E9125
:10626000EEDFF1DF708A800EE66E3EDAE552A00EB8
:10627000726E0E017D8F7D8D7D8B7D897D977D95E5
:106280000F0EF86F800EF96FFA69FB6BF70EE06F77
:106290007F0EE16F69C0E2FEE36BF70EE46F7F0EE5
:1062A000E56FE669E76BE8697F0EE96F69C0EAFEB2
:1062B000EB6BEC697F0EED6FEE69EF6B0F0EFC6F11
:1062C000E30EFD6FFE6BFF6B0F0EF06F820EF16F32
:1062D000F26BF36B79917993799579977999799BA9
:1062E000799D799F7A817A937A857A877A897A8B70
:1062F0007A8D7A8F7B817B837B857B877B897B8B88
:106300007B8D7B8F7C817C837C857C877C897C8B6F
:106310007C8D7C8F71917193719571977199719B3F
:10632000719D719F72917293729572977299729B1F
:10633000729D729F73917393739573977399739B07
:10634000739D739F74917493749574977499749BEF
:10635000749D749F75917593759575977599759BD7
:10636000759D759F76917693769576977699769BBF
:10637000769D769F77917793779577977799779BA7
:10638000779D779F78917893789578977899789B8F
:10639000789D789F46814683468546874689469BF9
:1063A000469D469F070E436FAC0E446F830E456FAC
:1063B0009DC2E6FF99D9E5523F0E72148009726EB4
:1063C000728AE00E72140509726E609E609C609A7B
:1063D000609860966094608260800E017E9F7E9DD2
:1063E0007E9B7E997E877E857E837E81769A769E51
:1063F0007682D08E78987896789478927890DCD15E
:10640000D6D9020EE1260201030E9F6F71AE83D032
:10641000070E6F14B009726E610EDE6E0F0EDD6E28
:10642000006A0D0E005C10E2DECFE9FFDDCFEAFF6F
:10643000EF50E66E0050EA6AA00FE96E020EEA2203
:10644000D1D9EFE3DB2AEDD7609E719E719EE00EFD
:106450000201A115E840E840E8401F0B006EA05182
:10646000070B070B200D030EA1150010F310A16FF1
:10647000A051080B18E1EE0EA15D15E10001695174
:106480000201A35D10E1A3514D6E4E6AFE0E4D1840
:1064900001E14E5008E0010E9F6F6F88719E719E62
:1064A000CEDED1DE0AD0A051080B06E1EA0EA15DD6
:1064B00003E1020E9F6F01D09F6B040E035C23E289
:1064C000032A022A040E025C01E3026A025078D910
:1064D000A0C2EEFFA1C2EEFFA2C2EEFFA3C2EEFF7A
:1064E000A4C2EEFFA5C2EEFFA6C2EEFFA7C2EEFF5A
:1064F000A8C2EEFFA9C2EEFFAAC2EEFFABC2EEFF3A
:10650000ACC2EEFF02D002019E8102019F0501E0B4
:106510007DD7719E719E9F514D6E020EE15C02E22D
:10652000E16AE552E16E4D5047D1065008E10E0197
:106530007F6B0F0E7E6F769802019C6B000C020140
:106540009C5106E09C0529D945D960B6020C9C6B8C
:106550000650000822E2060E9C5D1FE29C511DD9E8
:1065600039D960B617D004500D0DF3CF4DF0F4CFEC
:106570004EF0340E4D26020E4E224DC0E6FF4EC0A8
:10658000E6FF5DD8E552E552042A080E045C01E3FB
:10659000046A060602019C2BDBD79C05FED8080086
:1065A000F5CF7FFE9C05F9D8F62A000EF7220800E9
:1065B000F5500F090E017E6F7688000CF8D8080E92
:1065C000065C16E2062A052A080E055C01E3056A48
:1065D000A7D8ADD805500D0DF3CFE9FFF4CFEAFFF2
:1065E000340EE926020EEA22BDD802019F6B03D0C9
:1065F0000201010E9F6F76880E017F5105E1F00EBA
:106600007E1502E17F87778802019F51D5D0CFD8D0
:10661000769203500EE00150D3D889D881D8A2D801
:10662000012A040E015C01E3016A030602019F6B6B
:1066300003D00201010E9F6F76829F51BDD0B7D863
:10664000020EE1266DD8EF98D4D80F0EEF14000992
:10665000EF6ECFD8F00EEF140809EF6ED0D8E00B34
:10666000E838E8404D6E5CD84D50070BF36EF80EDD
:10667000EF14F310EF6EC3D8030B006EC0D81C0BE1
:10668000080DF350E66E4CD8EE52E552E750EF6E2F
:10669000080E00104D6E44D8EE524D50EF1260B609
:1066A000FED7610EDE6E0F0EDD6E006A0D0E005C11
:1066B00013E236D8E9CF4DF00050E924E96E000E20
:1066C000EA20EA6EEF50E66EDECFE9FFDDCFEAFFAB
:1066D00089D8ECE3DB2AEAD76086020EE15C02E2AD
:1066E000E16AE552E16E68D062D8FE0EDB506F6E53
:1066F000E00E6E144D6EFE0EDB504D5CF9E15CD089
:1067000056D8800EE66EF0DFE552FE0EDBCFE2FEDD
:10671000FE0EDBCFEAFE9DC2E6FFE6DFE5524CD07F
:10672000FD0EDBCFE9FFFE0EDBCFEAFF1200EECF5E
:106730004DF0EECF4EF0EECF4FF0EECF50F0EECF6B
:1067400051F0EECF52F0EECF53F0EECF54F0EECF4B
:1067500055F0EECF56F0EECF57F0EECF58F0EFCF2A
:1067600059F012004DC0EEFF4EC0EEFF4FC0EEFFDD
:1067700050C0EEFF51C0EEFF52C0EEFF53C0EEFF1F
:1067800054C0EEFF55C0EEFF56C0EEFF57C0EEFFFF
:1067900058C0EEFF59C0EEFF1200030DF3CFF6FF15
:1067A000F4CFF7FFF60EF626770EF7221200D9CFB8
:1067B000E6FFE1CFD9FF1200E552E7CFD9FF120083
:1067C0000D0DF3CFE9FFF4CFEAFF000EE926020E2C
:1067D000EA221200020EF626000EF7220800F550FB
:1067E000726E1200E552E750EF6E002ADF2A010EAA
:1067F000120096DF040EE926000EEA22120090DF56
:06680000EE52EF50120001
:0A6806000101030E6A6F010E6B6FB3
:10681000ED0E6C6F6D6969C06EF1736B750E6F6F05
:10682000010E706F746B74514D6E4E6A1B0E4D5C91
:10683000000E4E5809E27451EA6A750FE96E010EB6
:10684000EA22EF68742BEFD7746B120E106F010EF3
:10685000116F4E0E496F010E4A6F4B69060E006FA5
:10686000016BE80E026F036969C004F1070E056F42
:10687000010E066F060E236F246BEC0E256F266942
:1068800069C027F12A0E286F010E296F060E326F9C
:10689000336BEC0E346F356969C036F1390E376FE2
:1068A000010E386F060E416F426BEE0E436F446966
:1068B00069C045F1610E466F000E476F030E906F81
:1068C000010E916FED0E926F936969C094F19A0E6B
:1068D000956F010E966FD50E976F010E986F200E73
:1068E000D56F996B060EB56F010EB66FEE0EB76FD2
:1068F000B86969C0B9F1D60EBC6F010EBD6F200E2C
:10690000D66FBE6B060EBF6F010EC06FEE0EC16F6D
:10691000C26969C0C3F1C66BC76BC86BCA69030E95
:10692000CB6F010ECC6FF00ECD6F140ECE6F69C021
:10693000CFF1200ED76F860ED46F0501020E1E6FA9
:10694000010E1F6FF10E206F0D0E216F69C022F531
:10695000250E236F050E246F0501020E2D6F010E0B
:106960002E6FF10E2F6F0D0E306F69C031F5340EA2
:10697000326F050E336F0501020E006F010E016FBD
:10698000F20E026F036B69C004F5070E056F050E6A
:10699000066F0501020E0F6F010E106FF20E116FE0
:1069A000126B69C013F5160E146F050E156F0401F6
:1069B000020E4E6F010E4F6FF20E506F010E516FAF
:1069C00069C052F4580E536F040E546FD80E556FB1
:1069D000010E566F0101200E04011A0E576F0401BB
:1069E000020E726F010E736FF20E746F010E756FEF
:1069F00069C076F47C0E776F040E786FD80E796FCD
:106A0000010E7A6F0101200ED86F04011A0E7B6F00
:106A10000001020ECF6F010ED06FF20ED16F050E86
:106A2000D26F69C0D3F0D60ED46F000ED56F0001BF
:106A3000020EDE6F010EDF6FF20EE06F050EE16FEA
:106A400069C0E2F0E50EE36F000EE46F0301060E8D
:106A5000A26F010EA36FF20EA46F110EA56F69C095
:106A6000A6F3A90EA76F030EA86F0301060EB16F60
:106A7000010EB26FF20EB36F110EB46F69C0B5F3B1
:106A8000B80EB66F030EB76F0301060EC06F010E8E
:106A9000C16FF20EC26F110EC36F69C0C4F3C70E8F
:106AA000C56F030EC66F0301060ECF6F010ED06FC8
:106AB000F20ED16F110ED26F69C0D3F3D60ED46F20
:106AC000030ED56F0301060EDE6F010EDF6FF20EAF
:106AD000E06F110EE16F69C0E2F3E50EE36F030EA4
:106AE000E46F0301060EED6F010EEE6FF20EEF6F15
:106AF000110EF06F69C0F1F3F40EF26F030EF36F35
:106B00000401060ED66F010ED76FF20ED86F140E69
:106B1000D96F69C0DAF4DD0EDB6F040EDC6F04019F
:106B2000060EE56F010EE66FF20EE76F140EE86FCA
:106B300069C0E9F4EC0EEA6F040EEB6F0501020E7A
:106B4000536F010E546FFE0E556F100E566F69C0D5
:106B500057F55A0E586F050E596F29EC3BF034EC7F
:106B60003BF07FEC3BF089EC3BF0CAEC39F0EAEC0F
:106B700039F009EC3BF019EC3BF0D5EC38F0E3ECE4
:106B800038F0F1EC38F0FFEC38F00DEC39F01BEC9C
:106B900039F06BEC3BF075EC3BF0C2EC3BF00501DF
:106BA000256B0501010E346F0501076B0501010E10
:106BB000166F0401586B0401010E7C6F0001D66B47
:106BC0000001010EE56F0301A991A993A995A99769
:106BD0000301C791C793C795C7970301E591E59353
:106BE000E595E5970301B881B893B895B897030187
:106BF000D681D693D695D6970301F481F493F49574
:106C0000F4970401DD6B0401010EEC6F0401E46BE9
:066C10000401F36B120009
:0A6C1600D9CFE6FFE1CFD9FFFE0E53
:106C2000DB50266EFE0EDB50276E0001263A0F0E5B
:106C300026162650090802E2070E2626300E2626C2
:106C40000F0E27162750090802E2070E2726300EDE
:106C50002726E552E7CFD9FF120064D9FD0E87D968
:106C600003E0FE0E84D902E1FF0E27D0FE0E6FD99D
:106C700002E0300E01D0370E4D6EFE0EDBCFE7FF87
:106C80004D50E75EFE0EE7CFDBFFFD0E60D902E060
:106C9000300E01D0370E4D6EFD0EDBCFE7FF4D50AD
:106CA000E75EFD0EE7CFDBFFFD0EDB500F0B4D6EF9
:106CB000FE0EDB38F00BF00B4D1039D1300E2A6E82
:106CC000300E2B6E300E2C6E640E2D5C04E3640EC1
:106CD0002D5E2A2AF9D70A0E2D5C04E30A0E2D5EDA
:106CE0002B2AF9D7010E2D5C03E32D062C2AFAD7A7
:106CF000120043D90A0E2B02F3CF4DF0640E2A0284
:106D0000F3504D242C242D6E1200286A296A2A6A19
:106D10002B6A2C6A2E380F0BF00F296E2926E20FF2
:106D20002A6E320F2C6E2E500F0B2A262A262C2666
:106D3000E90F2B6E2B262B262D380F0B2B262C26FE
:106D40002B362C362C1E2C362D500F0B2C2629368C
:106D5000070E286E0A0E2B062C26D8A0ABEF36F0B5
:106D60002A062B26D8A0B0EF36F029062A26D8A06E
:106D7000B5EF36F028062926D8A0BAEF36F0300E47
:106D8000282629262A262B262C261200300E285E9D
:106D9000300E295EF2D82850536E546A100E5402F9
:106DA000F3CF54F0270E5302F3505426100E530223
:106DB000F3CF53F0F45054262950556E566AE80E1E
:106DC0005602F3CF56F0030E5502F3505626E80E46
:106DD0005502F45056265350F324516E5450562009
:106DE000526E2A50640D5150F3244F6E5250F420CD
:106DF000506E2B500A0D4F50F3244D6E5050F4201E
:106E00004E6E2C504D242F6E000E4E20306E120010
:106E100089D8ACA2FED7FE0EDB50AD6E88D082D8EA
:106E2000FE0EDB98DB9ADB9CDB9EFE0EDB50090836
:106E300002E2070E92D8300E90D8FE0EDBCFE6FFAE
:106E4000E7DFE55274D0ABD82D6E38DF2A50A3D8D7
:106E50002B50A1D82C509FD86AD064D80001FE6B6B
:106E6000FD0EDB50FE5D18E2FE0EDBCFE6FFE66AAC
:106E7000B7EC3AF0E552E5520001FF6FFE0EDB2A57
:106E8000FF0EFF5D02E12D0EFF6FFFC0E6FFC0DFCA
:106E9000E5520001FE2BE4D74AD044D8300E74D816
:106EA00004E3FE0EDB50390802E2000E01D0010EB1
:106EB0003ED038D8FE0E4BD809E1410E65D804E328
:106EC000FE0EDB50460802E2000E01D0010E2FD06C
:106ED00066D82B0806E0FE0EDB502D0802E0000EFF
:106EE00001D0010E24D05BD8500806E0FE0EDB5026
:106EF000530802E0000E01D0010E19D013D81BD8A0
:106F000010E0ACA2FED717D8AD6ED950FC0FE96ED9
:106F1000FF0EDA20EA6EEE2A000EEE22000EEE22BE
:106F2000EED705D0D9CFE6FFE1CFD9FF1200E55269
:106F3000E7CFD9FF1200FC0EDBCFF6FFFD0EDBCF53
:106F4000F7FFFE0EDBCFF8FF0800F5501200DBCF95
:106F5000E6FFA3DFE552000912004D6EFE0EDBCF07
:106F6000E7FF4D50E726FE0EE7CFDBFF1200DBCF39
:106F7000E6FF9FDFE55200091200300E2A5E300E58
:106F80002B5E300E2C5E1200F36EFE0EDBCFF4FF94
:106F9000F350F45C1200E66E3BDFE5521200C2DFF4
:066FA000FE0EDB501200A2
:0A6FA600205B6C74723D000D0A4977
:106FB0006E76616C696420436F6D6D616E643A003A
:106FC00053544E000D0A41363D20000D0A41353D17
:106FD00020000D0A41343D20000D0A41333D2000C0
:106FE0000D0A41323D20000D0A41313D200039207B
:106FF000536D616C6C4372616674202020202020E8
:1070000020202000382052756464657220202020E2
:1070100020200037204F696C204C6576656C20205D
:10702000200036205761746572204C6576656C20AF
:1070300000352042617474205374617475732000AC
:1070400034205472616E7320506172616D20003380
:10705000204675656C204C6576656C202000205BB1
:1070600070706C3D003220456E672044796E616D12
:1070700069632000205B7070723D003120456E67AF
:1070800020526170696420202000525331312076F3
:10709000002020203C4F66663E2020202000205407
:1070A00072696D2054616220202000205275646452
:1070B000657220506F73200020416C7420566F6CF5
:1070C0007473202000204F696C204C6576656C201D
:1070D000200020577472204C6576656C20200020BB
:1070E0004261747420416D707320200020547261DD
:1070F0006E732054656D702000205472616E732091
:10710000507265732000204675656C204C6576656D
:107110006C2000204675656C20507265732020003D
:1071200020436F6F6C205072657320200020436FE6
:107130006F6C2054656D70202000204F696C2054C6
:10714000656D7020202000204F696C20507265739F
:1071500020202000204261747420566F6C747320CC
:10716000002054696C742F5472696D2020002042F5
:107170006F6F737420507265732000284F66662904
:107180000020284F6E29005374626400506F72749F
:10719000000D0A4D657373616765000D0A00205389
:0971A0006E64725F4375727200A7
:0671AA000301A999A99B55
:1071B000A99DA99FAA697F0EAB6FAC69AD69AE6945
:1071C000AF69B06912000301C789C79BC79DC79FFC
:1071D000C8697F0EC96FCA69CB69CC69CD69CE69B0
:1071E00012000301E599E59BE58DE59FE6697F0EB9
:1071F000E76FE869E969EA69EB69EC691200030184
:10720000B899B89BB89DB89FB9697F0EBA6FBB6932
:10721000BC69BD69BE69BF6912000301D689D69BEE
:10722000D69DD69FD7697F0ED86FD969DA69DB6999
:10723000DC69DD6912000301F499F49BF48DF49F7D
:10724000F5697F0EF66FF769F869F969FA69FB6904
:0272500012002A
:0E725200396AE86A47AE36EF39F0446C451EE3
:10726000461E471E452246224722391E42AE41EFA6
:1072700039F03F6C401E411E421E402241224222F4
:10728000391EE5EC3AF042BE58EF39F039AE000C49
:107290003F6C401E411E421EE86A402241224222AB
:1072A0003B6C3C1E3D1E3E1E3C223D223E22000CFD
:1072B00039BE48EF39F03A88FF0C41C04BF04150DD
:1072C0004602F4CF40F0F3CF3FF042504702F4CFF4
:1072D00042F0F3CF41F04602F3504026F4504122F1
:1072E000E86A42224B504702F3504026F4504122B4
:0672F000E86A4222000CD6
:0A72F6002A0EF66E000EF76E000E71
:10730000F86E04010900F550F96F0900F550FA6FA5
:1073100003E1F96701D03DD00900F550F46F090091
:10732000F550F56F0900F550F66F09000900F550AA
:10733000E96E0900F550EA6E090009000900F550F0
:10734000F76F0900F550F86F09000900F6CFFBF45C
:10735000F7CFFCF4F8CFFDF4F4C4F6FFF5C4F7FF63
:10736000F6C4F8FF0401F75302E1F85307E00900FF
:10737000F550EE6EF707F8E2F807F9D7FBC4F6FF11
:10738000FCC4F7FFFDC4F8FF0401F907000EFA5B27
:04739000BFD7120051
:0C739400040159695A695B695C695D6914
:1073A0005E695F697F0E606F61697F0E626F6369FE
:1073B0006469656966696769686969696A697F0E90
:1073C0006B6F6C6B6D6B6E6B6F6B7F0E706F7F0E88
:1073D000716F120004017D697E697F69806981692E
:1073E000826983697F0E846F85697F0E866F8769E6
:1073F000886989698A698B698C698D698E697F0E54
:107400008F6F906B916B926B936B7F0E946F7F0E6F
:04741000956F120062
:0C741400D9CFE6FFDACFE6FFE1CFD9FFC9
:10742000E2CFDAFFE652DF6AFD0EDBCF4EF04EC050
:107430004DF0030E4E14756EFF0EE76EFC0EDBCFA3
:107440004DF0E7504D164E6A4D50746EFB0EDB50FA
:10745000736E7F9E7F9C7F84F250800B01E0010E53
:10746000DF6EF29E550E7E6EAA0E7E6E7F827FB21A
:10747000FED7DF50E8B0F28EE8A0F29E7F94E5528E
:0C748000E552E5CFDAFFE7CFD9FF12009C
:04748C00D9CFE6FF6F
:10749000DACFE6FFE1CFD9FFE2CFDAFFAC6AAB6A21
:1074A000FD0EDBB0AC88DBA202D0AC8CAB8CDBB4C5
:1074B000AC8EDBA602D0AB8801D0AB8ADBB8AC8443
:1074C000DBBAAB86DBAC02D09D8A01D09D9ADBAEE5
:1074D00002D09D8801D09D98FB0EDB50AF6EFC0E54
:1074E000DBCF4EF04EC04DF04E6A4D507D6EAC8AF3
:0E74F000AB8EE552E5CFDAFFE7CFD9FF1200F1
:0274FE003F50FD
:107500004402F3CF3BF0F4CF3CF04502F3503C266D
:10751000000EF4203D6E3F504602F3503D26000E13
:10752000F4203E6E3F504702F3503E264050440246
:10753000F3503C26F4503D22000E3E2240504502BE
:10754000F3503D26F4503E2240504602F3503E2672
:1075500041504402F3503D26F4503E224150450232
:0E756000F3503E2642504402F3503E261200E5
:02756E00D9CF73
:10757000E6FFDACFE6FFE1CFD9FFE2CFDAFFFC0E7C
:10758000DBCF4DF0FD0EDBCF4EF04EC04DF04E6A1E
:10759000030E4D14756EFF0EE76EFC0EDBCF4DF043
:1075A000FD0EDBCF4EF0E7504D164E6A4D50746E17
:1075B0007F9C7F9E7F8000000000735000D0E552CA
:0A75C000E5CFDAFFE7CFD9FF120094
:0675CA003E6A3D6A3C6AC6
:1075D0003B6A200EE76ED8903F3640364136423641
:1075E0003B363C363D363E3644503B5C45503C587D
:1075F00046503D5847503E5809E344503B5E455085
:107600003C5A46503D5A47503E5A3F2AE72EE4D74F
:02761000120066
:0E7612000001D785D787D789D78BD78DD78F23
:10762000D781D783D869D969DA69DB69DC6BDD6911
:1076300012000001E685E687E689E68BE68DE68F97
:10764000E681E683E769E869E969EA69EB6BEC6979
:02765000120026
:0E7652000501266927697F0E286F29697F0EC2
:107660002A6F2B692C6912000501356936697F0E76
:0E767000376F38697F0E396F3A693B69120037
:02767E003E6A62
:107680003D6A100EE76ED890413642363D363E36A2
:1076900046503D5C47503E5805E346503D5E4750DE
:0A76A0003E5A412AE72EF0D71200EF
:0676AA00D9CFE6FFDACFA4
:1076B000E6FFE1CFD9FFE2CFDAFFFD0EDB507C0B16
:1076C0004D6E830EC2144D10C26EE552E5CFDAFF47
:0676D000E7CFD9FF120014
:0A76D6000401DE697F0EDF6FE0693A
:1076E0007F0EE16FE269E36912000401ED697F0E2C
:0E76F000EE6FEF697F0EF06FF169F269120024
:0276FE00050184
:10770000086909690A690B697F0E0C6F0D690E69BA
:10771000120005011769186919691A697F0E1B6F34
:067720001C691D69120046
:0A772600D9CFE6FFDACFE6FFE1CF8E
:10773000D9FFE2CFDAFFFD0EDB50A76EE552E5CFB1
:08774000DAFFE7CFD9FF1200C8
:08774800410EF36E00EE00F0AB
:107750000E0E01D81200EA6002D0EE6AFCD7F35098
:08776000E9601200EE6AFCD79B
:087768001CEE00F02CEE00F015
:10777000F86A3A9C7BEC39F021EC3CF0CBEC30F031
:04778000FBD7120021
:0C77840005017F0E5A6F7F0E5B6F5C6981
:0C7790005D695E695F69606961691200F3
:04779C000803840456
:0E77A000038300839700439600239500139403
:0277AE000803CE
:1077B0008404038300839700439600239500139469
:1077C00008038404038300839700439600239500F5
:0277D000139410
:0E77D20008038404038300839700439600237A
:0477E0009500139469
:0C77E4000803840403830083970043968D
:0677F00000239500139434
:0A77F6000803840403830083970056
:08780000439600239500139448
:087808000803840403830083DC
:0A781000970043960023950013949F
:06781A000803840403834F
:0C7820000083970043960023950013940A
:04782C0008038404C5
:0E783000038300839700439600239500139472
:02783E00C28204
:02784000120034
:02784200120032
:0C78440024455252504D2C452C3F3F3F34
:107850002C3F3F3F3F2C2C410D0A002445525250F3
:107860004D2C452C3F3F3F2C3F3F3F3F2C2C410DA3
:107870000A0024504E4F4C412C3F3F2E3F3F2C3F9F
:107880003F2E3F3F2C3F3F2E3F3F2C3F3F2E3F3F61
:107890002C3F3F2E3F3F2C3F3F2E3F3F2C3F3F3F53
:1078A0003F3F3F3F3F2C3F3F3F3F3F3F3F3F0D0A62
:1078B0000024504E4F4C462C3F3F3F2C3F3F3F3F14
:1078C0000D0A0024504E4F4C462C3F3F3F2C3F3F6B
:1078D0003F3F0D0A0024504E4F4C452C523F3F2C49
:0678E0004E3F3F0D0A00BF
:020000040030CA
:0100000015EA
:0100010053AB
:0100020008F5
:0100030026D6
:010005008971
:010006008178
:010008000FE8
:01000900C036
:01000A000FE6
:01000B00E014
:01000C000FE4
:01000D0040B2
:00000001FF
